:10732300BEBCBEFDAEFD9F1E8EDE96BD9EBEA6BE3E
:10733300A6BEAEDEAEDEB6FEB6FEAF1EA6DE9E9DDA
:10734300A6BEAEBDAEBDA6BDA6BDAE9DAE9DC77F5E
:10735300D79FDFBFDFBFDFBFE79FE7BFD75DB6BC08
:107363009E9D8E5D7E3D7E1C7DFBB73EDFDFDF9FF6
:10737300DF9EDFBFD7DF869D65FC763E761F6DBD42
:1073830096BECFFFD7BEDFBECFDF867C4DBC4DDFC1
:10739300559D96DED7FFDF9EDFBF967E559D4DDD63
:1073A3005DDBB77EDF9EDF9FB69CAE7BD75EF7FFCC
:1073B300FFFFF7DEE79EDF7EC6DBD77ED7BFAE9D3E
:1073C300A63DA65EA65DAE5DB69EB6BEBF1FC75FF9
:1073D300AEDE8E5E965E967F969F967E967E8E3E00
:1073E300865E7E5E765E661D6E1D6E5E765F763EA3
:1073F300763E867E96BE969E9E9E9E9E9EBEA6BF11
:10740300A6BFA6BFA69EA69EA69E9E5DA67DA67EA1
:10741300A69EA69F9E9E9E9F969F969F967E8E7EDD
:107423008E7E967E967E969E9EBE9EBFA6BFA6DF4E
:107433009EDF9EDF96FF9EFE9EDE9EDE9EBF9E9E8D
:107443009E9E96BF8E9F969F9E5E865F867F8E5E74
:10745300965E9E7F9E9F9E9F969F969EAEBECF5F9B
:10746300CF7FA6BE7E5E6E3E5E1E561E561E561E07
:107473004E1E4E1F4E1F461F4E1F4E1F4E1F4E1FAA
:107483004E1F461F463F4E3F4E1F4E1F4E1F4E1F61
:107493004E1F561F4E1F463F463F4E3F4E1F4DFF4A
:1074A3004DFF4E1F4E1F4E1F4E1F4E1F4E1F4E1F92
:1074B3004E1F4E1F461F4E1F4DFF4DFF4DFF45FFF5
:1074C30045FF45FF4DFF4E1F563F5E3F5E5F665FC4
:1074D3005E3F561F4E1F4DFF4DFF4DFF4DFF4DFFAE
:1074E3004DFF4DFF4DFF4DFF4DFF4DFF4DFF4DFF39
:1074F3004DFF4DFF4DFF4DFF4DFF4DFF4DFF4DFF29
:1075030043B44CB95D7D6DBBCF7FF7FFFFFFFFFF3A
:10751300FFFEFFFFFFFFFFDFF7DFE7FF8E7D559CD9
:107523005E1E65FE761E7E3E7E5F863E963DDFBF17
:10753300EFFFF7FEFFDEFFBFF7BFF7DFEF9FCEFEE4
:10754300BEDFAEBFB6BFBF1FAEFFBEFEEFDFF7BEEF
:10755300F7BEEFBEEFFFAF7F559C55DE4DFF4DDE0F
:1075630065DCBF5EE7DEEF9DDFBEBF9F6E1D55FE90
:107573005DFD6E1BB77FCF9FCFBEBFBF8E9D7E3D90
:10758300965CC6FDEFDFEFDFF7FFFFFEFFBEFFBE3A
:10759300F7DFF7FFFFDEFFFFEF9EE77ED77ECF5FCC
:1075A300BF1FBF1FBEFFBEFFA67EA67EAEBFA69EA9
:1075B3009E5DA69EA6BEAEDEA6BE9E7D9E7E9E7EE2
:1075C3009EBE9EBE9EFE9EDE96BD9EDE9EDE9EBE41
:1075D300969E9EBEAEDFB6DEB6FFB6FFB6FFAEDF4B
:1075E300AEDFAEFFAEFFAEFFAEFFAEDFAEDFA6DFB8
:1075F300A6BF9EBF9EBF96BF969F969F967F9E9F58
:10760300A6BFA6BE9EBE9EBE9EBE969E869E763E8E
:10761300661D5E1D5E1E5E1D5E1D5E1D5E1D6E5D36
:10762300663D563D563E5E1E6DFD761D75FC8E5DB8
:10763300A6FF96DF869F6E7F663E867E9EFF9E9F99
:107643007E1D5DFD561E4E1E4E1E4E3E4E3F4E3F50
:107653004E3F4E3F4E3F463F4E3F4E3F4E3F4E3FC7
:107663004E3F4E3F4E3F4E3F561F4E3F4E3F4E3FC7
:107673004E3F4E3F4E3F4E3F463F4E1F461F461F17
:107683004E1F4E1F4E1F4E1F4E1F4E1F4E1F4E1F8F
:107693004E1F4E1F4DFE4E1F561F55FE5DFE5DFED7
:1076A30055FE4DFE4E1F4DFE4DFE561F4DFF4DFE2A
:1076B30055FF4DFF4DFF4DFF4DFF4DFF4DFF4DFF5F
:1076C3004DFF4DFF4DFF4DFF4DFF4DFF4DFF4DFF57
:1076D3004DFF4DFF4DFF4E1F4E1F4E1F4E1F4DFFC3
:1076E30095BA54155C779E3DDF7FF7DFF7DEF7DE53
:1076F300F7DEF7BEF7DFF7DFF7BEF7DFAEBD5DDD21
:10770300561F561F5DFF6E1F6E3F661F7DFDB71E22
:10771300E7FFEFDEF7DEF7BFF7BEEFDFEFDFBEBD5C
:10772300A65DA67DA69DAEBDAE3CAE3BD79FD7DF83
:10773300CFBFCFBFD7BFB75F8E9D8EBD86DE86DE40
:107743008E9DAEFEB71FAF1FA6DEA69DB75EBF5EC2
:10775300BF5EC77E9EBD7E1C865C9E9CC73EE79F28
:10776300EFBFF7BEFFBDF7DFEFBFF7BFFFDFFFDF01
:10777300FFDFFFDFFFDEF7DEFFFFEFFFD73EBEFEDB
:10778300BF3EB71FB6FEAEBEA67DAEDEAEBE9E5DED
:10779300A67DAE7CBEFDD77FCF7EC71DC71EC73F6C
:1077A300CF3FCF1EC6FEC71FC73FC71FC71FC73F59
:1077B300C73FC71FC73FCF3FC71FC71FC71FBF1F36
:1077C300B6FFB6FFB6FFAEFFAEDFAEDFA69EA69E48
:1077D300A69EAEBEAEDFAEDFA6BEA6BEAEBFAEDF1A
:1077E300AEFFAEFEA6FFA6FF96BF7E5E6E5F665E31
:1077F300563F4E3F4E3F563F563F65FCA6FDBFBF2B
:10780300869C65DA863CAEFEC75FD77FCF3ED77FC7
:10781300C77F9E9E7E1D6E3E5DFD6DFD7E3E75FEA9
:10782300661E563F4E3F463F4E1F4E1F4E1F4E1F76
:107833004E1F4E1F4E1F4E1F4E1F4E3F4E3F4E1F9D
:107843004E1F4E1F4E3F4E3F4E3F4E3F4E1E4E1E4F
:10785300463E3E3E465E563E5E3E665E6E5E6E5EF5
:10786300665E5E3E4E3E4E3E4E3E4E1E4E1E4E1ECD
:107873004E1E4E1E4E1E5E3F667F6E9F767F6E7F50
:10788300663E561E4E1F4E1F4DFF4DFF4DFF4DFFD3
:107893004DFF4DFF4DFF4DFF4DFF4DFF4DFF4DFF85
:1078A3004DFF4DFF4DFF4DFF4DFF4DFF4DFF4DFF75
:1078B3004DFF4DFF4DDE55DE55DE55BE4DDF4DFF11
:1078C3009578955784B49D16E75EFFFFF7DFFFDFDA
:1078D300FFFFFFFFFFFFFFFFF7DFF7FFCF3E965DE1
:1078E300763D661D6E1D761D763D7E5E861CA6DD8D
:1078F300D79FDF5FE77FE77EEF7FEF9FEF9FE7BFD6
:10790300DF7ED75ECF3ECF5EC73DC75EA6DD7E1C62
:10791300661D663D6E1C6DDBA71DE7FFF7DEF7BE38
:10792300EFFFC79F7E1D763E867F8E5DCF7FEFFF85
:10793300EFBFEFDFCF9F9E9D9E7E9E9EB6DDDFBF96
:10794300F7BFFFBFFFDEFFDFFFDFFFDFFFDFFFDF8D
:10795300FFFFFFDFFFBEF7BDEFBEE79ECEDDDF5EBD
:10796300DF9EB6DDB6DDD75ED73DE7BFDF9FCF5ED7
:10797300D77ED75EEFFFF7FFFFFFFFFFF7DEF7FFCF
:10798300F7DFEFBFDF5EDF7ECF1EBEFEB6DDB6DE06
:10799300B6FEBF1FBF1FBF1FBEFEBEFEBEDEBEFFC5
:1079A300B71FB6FFB6FFB6FFBF1FB6FFB6DEB6DD25
:1079B300B6DEBF1EC73FC73FC73FC71EBEFEBEDE04
:1079C300B6DEB6FFAEFF969E7E5E767E765E6E5E1A
:1079D3006E7E6E5E6E5E6E5D6E5D7DFACF3ECF5FD8
:1079E3008E5B8E9BCF7FF7DFEFDFEF9FE77FD75F66
:1079F300B6BD9E7D9EBF867E863D967E9EBF9EDFE4
:107A030096DF869E765E6E7F6E7F667E667F665E9F
:107A13005E5E5E7E5E7E5E7E5E5E5E5E5E7E567FEA
:107A2300567F565F565E563E5E5E6E3D869E8EBEAA
:107A3300869E7E9F76BF767E7E9E867E8E7E867EA9
:107A4300767E665D565D563E5E3E5E3E5E3F563ECC
:107A5300563E565E563E5E3E5E3E5E5E5E5E563E03
:107A63005E3E565E4E5E563E563E561E563E563E53
:107A73004E3E563E563E563E563F4E1E4E1F4E1FE0
:107A8300561F561E561E563E4E3F563F563F561FD6
:107A93005DFD763D96DEA6FEA6FF96BF7E7E663F23
:107AA300BE5ABE5ACE9BADB89D15BE3AE7BFDF5E48
:107AB300D73ECF3EC6FEBEDEB6BDBE9DCF1EDF9F08
:107AC300D79ECF7ED79ED79EDFBFE7BFE7DFDF7EA0
:107AD300BE5CBE5DBE9EC6DFCEDED6FEC69DD6FDB7
:107AE300F7DFF7DFFFDFFFFEFFFFF7FFCF7F861C28
:107AF300763E661F65FE7DDCAEBCE7DFEF9EF7BF1B
:107B0300EFDFDFFFA6DE7E1D863E965DAEBCDF9F08
:107B1300DF9ED77ECF7EBF5EC75ECF3ED75EEFBF11
:107B2300FFDFFFBFFFDFFFDFFFDFFFDFFFDEF7DF8B
:107B3300F79FEF9FF7FFF7FFEFDFD6FDCEDDE79F60
:107B4300EFDFE79EEF9FF7DFFFFFFFFFF7DFF7DFD3
:107B5300EFDFEFDFEFBFF7DFFFDEFFDEFFFFFFDF6C
:107B6300FFDFF7BFF7BFF7BFE79FE7BFD75EC6FDEE
:107B7300B6DDB6FDBF1EBF3EBF3EBF1EBF1EBF1E4E
:107B8300BEFEBEFEBEFEBEFEC71EC71EC73ECF5F05
:107B9300CF7FCF5FCF3ECF3EC71EC71EC71EBF1EC0
:107BA300BF1EBF1EAEFDA6DD9EBC9EDD9EFDA6FDD7
:107BB300A6FD9E9CAEFDBF5ECF5ED77EDF5EDF7E01
:107BC300CF9FAEDCC6FDE77FDF5ECF3ED77EBEFD37
:107BD300B6FDBF1EBF3EB6FEB6FEB71EAEFEAEFD81
:107BE300A6BCA6BCA6DD9EDD96BC96BC96DD96BD66
:107BF3008EBC8EBC8EBD8EBD8EBC86BD86BC86BC47
:107C030086BC8EBC8EBC96BCA6DDAF3EB75EB71DF0
:107C1300B6FDAE9CAE9C9EBC9EBC9EBC8E5B965C31
:107C2300AEFDB71EAEFEA6FE96DD7E9C7EBD76BD86
:107C33007E9D7E9D769D769D769D769D769D769D99
:107C4300769D769D7E9D86DD86BD86BE7EBE769DB7
:107C53006E9D6E9D6E9D6E9D6E7D6E7D6E7D6E7D49
:107C63006E7D667D667D667D667D667D6E5C769DDA
:107C7300A71EBF3FB6FEBF3FB73F9EFE86DE769E82
:107C83008D168D168CF68D169538324D5BD39DDB94
:107C930095FC8DDC85DD7DFE861E85FD9E3DE7BF63
:107CA300FFFFFFDEFFDEFFFFFFDEFFDDFFDEEFBFD7
:107CB300B65DA63EA67F9E5FA65EAE7EAE5DB65B5C
:107CC300E79EF7DFF7DEFFDEFFDEF7DFDFBFAE9D08
:107CD300A69DA6BFAEFFCF5FDF9FE7BFEFBFEFBF9E
:107CE300EFDFE7BEDFBFD77FCF5FDF9FE7BFE79E53
:107CF300CF1DBEFDAE7CBEDCE7DFF7FFFFDFFFDE9F
:107D0300F7BFF7BFFF9FFFBFFFDFF7DEF7FFE77E9A
:107D1300D6BDD6DDDF5FDF9FD77ED75EDF5DEF9F0A
:107D2300EF7EF7BFFFDFF7BEFFBEFFDFF7BFEFBF9B
:107D3300E77FEF7FEF9FF7BEFFBEFFBEFFBFF7BF3B
:107D4300F7BFF79FEF9FE75EDF3EE79FEFBFDF9F42
:107D5300C73FC73FC73FC73FBF1EC71FBF1FBF1F89
:107D6300B6FFB6DEB6DEB6DEB6DEB6DEB6DEAEDF56
:107D7300B6FFB6DEAEBEAEBEB6BEB6DFB6FFAEDF94
:107D8300B6DFAEBEAE9DAEBDB6BDC73EE7BFE79F95
:107D9300CF1DCEFCDF5EEFBFF7DFFFDFF79EE77E91
:107DA300E7BFC6DDBE9DC6FEC6BDB6BEAEBE9E7DEA
:107DB300967D967D965D967E8E5E8E3E8E1D8E3D65
:107DC3009E7D9E7DA69DA69D967D969D8E5D7E1C29
:107DD3007E3D8EBE869E7E3E761E763E763D763D0B
:107DE3007E5E865E969EAEBFAEBF9EDF8E9E7E5C3F
:107DF30075FB7E3CA6BEBEBEBEDFAEFF9EBE9EBE74
:107E0300AF1EB6DEA6BE8E9E765D563D4E5D4E3DE2
:107E13004E1E55FE4E1E4E1E4E1E4E3E4E3E4E1DD9
:107E23004E3E5E1D6E3D767E7E7E765E663E5E1DBA
:107E3300561D561D561D561E561E561E55FE5E1EBB
:107E43005DFF5DFE5E1E5E1E661E6E1E6DFE7E3E49
:107E5300867E863E7DFD75DC6DDC5DBC55DD661E74
:107E630063F4641474766C55957A4331222D2AB0E9
:107E7300649785FE7E1E75DE75FE75DE963DD79F83
:107E8300F7DEFFDEFFDFF7DFF7DEF7DEF7FFE7FF03
:107E9300BEDEA67EA6BF9E7EAE7EB6BEB6BEBEBD0F
:107EA300D75EDF9EDF9FDF7FD75ECF3FC71ED73E04
:107EB300E79EF7BEF7BFF7DFEFDFE77ED71EDF3FB3
:107EC300E75EE75DE75DFFBEFFFFFFFFFFFFF7DF55
:107ED300E7BFC71EBEDED73EEFBFFFFFFFDFFFDFFB
:107EE300FFDFF7DFF7BFF7BFF7DFEFBFE79FD71E70
:107EF300DF7FE79FDF5EBE9DAE5DBEBDE7DFF7DFE1
:107F0300F7BFF79FF7BFEFBFEF9FE77FDF5FD73F76
:107F1300CEFEDF3FEF7FF7BFF7BEEF9EEF9FE77F1A
:107F2300DF7FD73FC6FEC6BEC6FFC71FC73FBEFE25
:107F3300B6DFBEFFBF1FBEFFB6FFB6FFB6FFAEFF85
:107F4300A6FFA6DFA6DFA6DFA6DFA6DFA6DF9EBF0E
:107F53009EBF9EBF9E9FA6BFA6DFA6BFA69EA69E50
:107F6300AEBFA69EAE9EBEDED77FE7BFEF7FEF5FBD
:107F7300EF7FEF9FE77FE75EE77EEF7EEF7EDF7EBB
:107F8300DF5FDF5FC75FBF3FAE9EA69F969F969F53
:107F93008EBF869E7E7E869F867EA6BEB73FC75FC8
:107FA300CF9FCF5FCF3FCF5FD77FCF5FCF5FBEFE88
:107FB300BF1FB73FAEDF9EDF8EDF8EBF86BF86BF9C
:107FC300869E867E8E9F867E867E869E7E9E867E0D
:107FD300967EAEFFB6FFC6DFB6BFA69EA6FF96FE91
:107FE3008E9D8E7C8E5D8E5E7E7E767E6E9F6E9F78
:107FF3006E7F6E5F6E5E6E7E665E663E665E665E1C
:108003006E7F6E7E6E5D6E3D6E3D6E5E6E5E6E7EEF
:10801300667E6E7F6E5E6E5E6E5F6E5F6E3F6E5FE0
:108023006E5F765F767F769F769F767F7E7F7E7F9D
:108033007E7F7E9F7E9F7E9F7E7E7E7F867F8EBF9E
:1080430084D784B663927C55ADDB4B303ACF2A8E0E
:108053001A4D3B52757B865E8E5E965FAE9DD79FB3
:10806300F7FFF7DFF7DFF7DFEFDFDF9FDF9ECF5E9F
:10807300BEDDBEDDC6FDD73EDF7EE79FE79EE7BFE1
:10808300CEFDAE3CB69EAE7E9E5D9E9F8E1DBEFE19
:10809300F7FFFFBEFFBEFFDEFFFFE79FC6BEC6DEE4
:1080A300D73EEF7FEF9FF7BEF7FFF7DFFFDEFFBEA1
:1080B300EF7ED71EDF7FEFBFEFBFE77EDF3EE75FD9
:1080C300E77FF7DFF7DFF7DFE7BFC6DEBE7DB65C2E
:1080D300D77FE7DFE7DFBEBDA63DB69DCF5EDF7E80
:1080E300F79FF7BFF7DFE79FD73ECF3FC71FC6DF37
:1080F300C6FFCEFFD73EDF7EE79EE7BFD73EBEBEBD
:10810300AEBE9E7E9E5E9E5F9E7F9E7F9E7E9EBF38
:108113009E9F9E9F9EBF9EBF969E969E969E9EBE30
:10812300A6BEA6BEA6BEA6BEA6BEA6DEA6BEA6DEEC
:10813300A6BE9E9E9E7DA6BFAEDFA69EA69EA6BEA3
:10814300AEFFA6BFAEBFBEFFC6FECF1ECEDDC6DDF1
:10815300CF1ECF1FD71FDF1EE75EE75FD73FBEFDF2
:10816300C6DEC6DFAEFF9EBF9E7F967E969E8E9E28
:108173008EBF8EBF8E9F96BF96BFA6DFB71FB6FF7B
:10818300B6DEBEDFBEDFBEDFBEDEBEFFB6FEAEFFC7
:10819300A6DF965D8E7E8E9E869F869F7E9F7E9FA8
:1081A3007E9E7E9F7E7F769E7EBF7E7F867F8E7F36
:1081B300969FA6BE9E9D8E9E969E9E9E9EBFA6BF8A
:1081C300AEDFAEFFAEFFAF1FAF1FB71FAEFFAEFFF9
:1081D300AEFEA6FEAEFFAF1FAEFFAEFFAEFFAEFF1D
:1081E300AEDFA6FF9EFFA6DFA6BFA6DFA6BF9EBF8C
:1081F3009EBF9EBF96DF96BF8EBF86BF869E7E9E26
:10820300765E765F6E5F6E5E665E663E661E6E3F90
:108213006E5E6E5E6E5E767F765E765E7E7E7E5E82
:10822300533042AE0886426D8C956BD263F36C7506
:108233004B921A2D32F08DBBA69EBEDDC6FDD75ED6
:10824300DF5EDF3EDF3EDF3DD71DC69DBE9CAE3BFE
:10825300BEDDEFFFF7FFFFFFFFFFFFDFFFFFF7FFCE
:10826300D73EAE7DAE9F963E8E3F863F85FDA65D93
:10827300E7BFF7DFF7DFF7DEF7DEEFDFC6DDBE7D53
:10828300CEDDDF1DE73EE77EE7BFE7BFE79FEF7E7B
:10829300F7BFF7FFF7DFF7DFEFFFC6BCBE5CC6BE75
:1082A300BE9DDF7FEFDEEFDFDF9FB65CAE3CAE1B34
:1082B300B6DDC73EBEFEB6BECF3FDFFFCF7DCEFDF0
:1082C300DF3FEF7FF7DFE79FCF1EC6FFBEDFB6BE00
:1082D300BEBEBEBECF3FDF7FDF9FE7BFCEFDB63B57
:1082E300961D8E3E8E3E8E3E967F969F9EBF9EBF70
:1082F3009EBE9EBF9EBF9EBF9EBE96BE9EDFAF1F0D
:10830300B71FBF3FBF5FBF3FC75FC75FC73FC73F22
:10831300C75FC75FC75FBEFEB6DFB6DFB6DFB71F97
:10832300AEDFAEDFB6FFBEDFC6FEC6FEC71EC71E8C
:10833300BEFEC6FFCF1FDF5FE77FDF5FC73FAEBE77
:10834300A65CAE9E9E7E8E7E967E969D969D8EBEEE
:1083530096DE96BE969E9E9F9EBF96BF969F969FC5
:10836300967E965E967F967F967E967E8E5E8E5ED8
:10837300865E869F869F869F8E7E8E7E867E867E87
:10838300867E869E869F7E9E7E9E7E7E867E867E61
:10839300869E7E7D86BE86BF869F8EBF8EBF8E9F46
:1083A3008EBF86BF8EBF8EDF8E9F969F8E7E8E5E24
:1083B300865D7E5D865D865D8E9E96BE9EDF9EFF9C
:1083C30096DF96DF96DF96BF96BF969F9E9F9EDFB2
:1083D3009EDFAEBFAEDFAEDFA6DFA6DF9E9F8E7F42
:1083E300865F765F6E5F663E663E663E663E6E1FE6
:1083F300661E663F6E5F6E7F665E665E6E5E6E3E97
:1084030007E007E007E007E007E007E007E007E031
:1084130007E007E007E007E007E007E007E007E021
:1084230007E007E007E007E007E007E007E007E011
:1084330007E007E007E007E007E007E007E007E001
:1086730007E007E007E007E007E096B6BE3A773287
:1086830007E007E007E007E007E007E007E007E0AF
:1086930007E007E007E007E007E007E007E007E09F
:1086A30007E007E007E007E007E007E007E007E08F
:1086B30007E007E007E007E007E007E007E007E07F
:1086C30007E007E007E007E007E007E007E007E06F
:1086D30007E007E007E007E007E007E0478DB5FAAA
:1086E300ADF9C61AB679675107E007E007E007E07E
:1086F30007E007E007E007E007E007E007E007E03F
:1087030007E007E007E007E007E007E007E007E02E
:1087130007E007E007E007E007E007E007E007E01E
:1087230007E007E007E007E007E007E007E007E00E
:1087330007E007E007E007E007E007E007E007E0FE
:108743007EF3BDDAADF9ADF9B5F9C61BAE98576F37
:1087530007E007E007E007E007E007E007E007E0DE
:1087630007E007E007E007E007E007E007E007E0CE
:1087730007E007E007E007E007E007E007E007E0BE
:1087830007E007E007E007E007E007E007E007E0AE
:1087930007E007E007E007E007E007E007E007E09E
:1087A30007E007E0AE58B5D9ADD9ADD9ADD8ADF92D
:1087B300B5D9C5FB9ED63FAD07E007E007E007E06C
:1087C30007E007E007E007E007E007E007E007E06E
:1087D30007E007E007E007E007E007E007E007E05E
:1087E30007E007E007E007E007E007E007E007E04E
:1087F30007E007E007E007E007E007E007E007E03E
:1088030007E007E007E05F4FBDFAADD9B5D9B5D9A9
:10881300ADF9ADD8CEBBC67ABDB9C61A8EF42FABAF
:1088230007E007E007E007E007E007E007E007E00D
:1088330007E007E007E007E007E007E007E007E0FD
:1088430007E007E007E007E007E007E007E007E0ED
:1088530007E007E007E007E007E007E007E007E0DD
:1088630007E007E007E007E007E08EB5B5DAADF90A
:10887300ADD9ADD9B5F9ADD8D6BBF7DFE73CBE1955
:10888300BDDAB6597F1207E007E007E007E007E02B
:1088930007E007E007E007E007E007E007E007E09D
:1088A30007E007E007E007E007E007E007E007E08D
:1088B30007E007E007E007E007E007E007E007E07D
:1088C30007E007E007E007E007E007E03FACBE1979
:1088D300ADD9B5D9ADD9ADD9ADD9ADD9ADB8BE192D
:1088E300E73DFFDFD6FCB5F9C5FBBE796F5107E065
:1088F30007E007E007E007E007E007E007E007E03D
:1089030007E007E007E007E007E007E007E007E02C
:1089130007E007E007E007E007E007E007E007E01C
:1089230007E007E007E007E007E007E007E007E00C
:108933007712BDDAADD8ADD9ADD9ADD9ADD9ADD9F1
:10894300ADF9ADD8ADB8C65ADF1CADF9ADF9B5FA7E
:10895300C61BAE98478D07E007E007E007E007E096
:1089630007E007E007E007E007E007E007E007E0CC
:1089730007E007E007E007E007E007E007E007E0BC
:1089830007E007E007E007E007E007E007E007E0AC
:1089930007E007E0A657B5D9ADF8ADD9ADD9ADD944
:1089A300ADD9ADD9ADD9ADF9ADF9ADD8ADB8ADD976
:1089B300ADD9ADD9ADF9BDFAAE3807E007E007E0B0
:1089C30007E007E007E007E007E007E007E007E06C
:1089D30007E007E007E007E007E007E007E007E05C
:1089E30007E007E007E007E007E007E007E007E04C
:1089F30007E007E007E0576FBDDAADD9ADF8ADD9B1
:108A0300ADD9ADD9ADD9ADD9ADD9ADD9ADD9B5F90B
:108A1300B5F9ADD9ADD9ADD9ADF8AD98963507E077
:108A230007E007E007E007E007E037A96EC907E0C2
:108A330007E037A907E007E007E007E007E007E002
:108A430007E007E007E007E007E007E007E007E0EB
:108A530007E007E007E007E007E08EB4BDDAADF911
:108A6300ADD8ADD9ADD9ADD9ADD9ADD9ADD9ADD9D4
:108A7300ADD9ADD9ADD9ADD9ADD9ADD9ADD8B5781D
:108A83005F0F07E007E007E007E007E007E0CE2419
:108A93008E4707E0966607E007E007E007E007E098
:108AA30007E007E007E007E007E007E007E007E08B
:108AB30007E007E007E007E007E007E037ACB61997
:108AC300ADD9ADF9B5D9ADD9ADD9ADD9ADD9ADD94B
:108AD300ADD9ADD9ADD9ADD9ADD9ADD9ADD9ADF943
:108AE300ADB8ADD707E007E007E007E007E05F09AF
:108AF30007E0BD649CA56728F5025E8807E007E0F0
:108B030007E007E007E007E007E007E007E007E02A
:108B130007E007E007E007E007E007E007E007E01A
:108B23006F11BDDAADF8ADD9ADD9ADD9ADD9ADD9E8
:108B3300ADD9ADD9ADD9ADD9ADD9ADD9ADD9ADD902
:108B4300ADD9ADF9B5797E9307E007E007E007E01B
:108B53009EA68E6707E075C807E04749AC6436C830
:108B630007E007E007E007E007E007E007E007E0CA
:108B730007E007E007E007E007E007E007E007E0BA
:108B830007E007E0A677B5DAADD9ADD9ADD9ADD950
:108B9300ADD9ADD9ADD9ADD9ADD9ADD9ADD9ADD9A2
:108BA300ADD9ADD9ADD9ADD8AD98476D07E007E0E4
:108BB30007E007E0C5C5CC6307E007E007E0470926
:108BC30007E007E007E007E007E007E007E007E06A
:108BD30007E007E007E007E007E007E007E007E05A
:108BE30007E007E007E0476DBDFAADF9ADD9ADD9B0
:108BF300ADD9ADD9ADD9ADD9ADD9ADD9ADD9ADD942
:108C0300ADD9ADD9ADD9ADD9ADF9AD989E3607E0A3
:108C130007E007E03FA907E085A83E6807E0A685CF
:108C2300AE0607E007E007E007E007E007E007E03C
:108C330007E007E007E007E007E007E007E007E0F9
:108C430007E007E007E007E007E086D4BDDAADD828
:108C5300ADD9ADD9ADD9ADD9ADD9ADD9ADD9ADD9E1
:108C6300ADD9ADD9ADD9ADD9ADD9B5D9ADF9B57901
:108C730066F007E007E05F476EA807E0378A07E082
:108C830007E0A606CC2307E007E007E007E007E0DC
:108C930007E007E007E007E007E007E007E007E099
:108CA30007E007E007E007E007E007E02FCBB6188F
:108CB300ADD9ADF9B5D9B5D9B5D8B5D8B5D8ADD83D
:108CC300ADD8ADD8ADD8ADD8ADD8ADD8ADD8B5D871
:108CD300ADD8ADD737AB07E007E0DDE4B58507E0F6
:108CE30007E066E82FAA6E082EE907E007E007E031
:108CF30007E007E007E007E007E007E007E007E039
:108D030007E007E007E007E007E007E007E007E028
:108D13006F11BDDAADD8ADD8B5D8B5D8B5B8B5D81B
:108D2300B5B8ADD8ADD8ADD8ADD8ADD8ADD8ADD830
:108D3300ADD8ADD8B598869307E007E007E0A56600
:108D43007D0507E06F27CDC407E007E007E007E0F4
:108D530007E007E007E007E007E007E007E007E0D8
:108D630007E007E007E007E007E007E007E007E0C8
:108D730007E007E09E56B5D9ADD8ADD8ADD8ADD88C
:108D8300ADD8B5D8B5D8ADD8ADD8ADD8ADD8ADD8A8
:108D9300ADD8ADD8ADD8ADD8B578574E07E007E01C
:108DA300378A5EAA07E007E076E8E4024E8907E027
:108DB30007E007E007E007E007E007E007E007E078
:108DC30007E007E007E007E007E007E007E007E068
:108DD30007E007E007E0478DBDF9ADF9B5D9ADD997
:108DE300ADD9ADD9ADF9ADF9ADF8ADD9ADD9ADD9F1
:108DF300ADD9B5F9ADD9ADD9ADF8ADB895F507E0B5
:108E030007E007E007E007E007E007E066895608A8
:108E130007E007E007E007E007E007E007E007E017
:108E230007E007E007E007E007E007E007E007E007
:108E330007E007E007E007E007E08ED4BDDAA5B856
:108E4300ADB8B5F9ADD9ADD9B5F9B5F9ADD9ADD998
:108E5300ADD9ADD9ADD9ADD9ADD9ADD9ADD9B57937
:108E63006EF107E007E007E007E007E007E007E04F
:108E73002F8A07E007E007E007E007E007E007E0E5
:108E830007E007E007E007E007E007E007E007E0A7
:108E930007E007E007E007E007E007E007E0AE3898
:108EA300B5D98CB4A577B5F9ADD9ADD9B5D9B5D9FF
:108EB300B5D9ADD9ADD9ADD9ADD9ADD9ADD9ADD977
:108EC300ADD9ADB837AC07E007E007E007E007E04E
:108ED30007E007E007E007E007E007E007E007E057
:108EE30007E007E007E007E007E007E007E007E047
:108EF30007E007E007E007E007E007E007E007E037
:108F03005F30C5DAADD894D5B5D9ADD9ADD9ADD922
:108F1300ADD9ADD9ADD9ADD9ADD9ADD9ADD9ADD91E
:108F2300ADD9ADF9B599867407E007E007E007E02E
:108F330007E007E007E007E007E007E007E007E0F6
:108F430007E007E007E007E007E007E007E007E0E6
:108F530007E007E007E007E007E007E007E007E0D6
:108F630007E007E09E96B5FAA577A577B5F9ADD9E1
:108F7300ADD9ADD9ADD9ADD9ADD9ADD9ADD9ADD9BE
:108F8300ADD9ADD9ADD9ADD8B598574F07E007E006
:108F930007E007E007E007E007E007E007E007E096
:108FA30007E007E007E007E007E007E007E007E086
:108FB30007E007E007E007E007E007E007E007E076
:108FC30007E007E007E03F8DBDFAADF98CD4ADB8FB
:108FD300B5F9ADD9ADD9ADD9ADD9ADD9ADD9ADD936
:108FE300ADD9ADD9ADD9ADD9ADF9ADB9A5F607E0D8
:108FF30007E007E007E007E007E007E007E007E036
:1090030007E007E007E007E007E007E007E007E025
:1090130007E007E007E007E007E007E007E007E015
:1090230007E007E007E007E007E07EF3BDDAA59776
:1090330094F5B5F9ADD9ADD9ADD9ADD9ADD9ADD9D2
:10904300ADD9ADD9ADD9ADD9ADD9ADD9ADF9B57925
:1090530076D207E007E007E007E007E007E007E074
:1090630007E007E007E007E007E007E007E007E0C5
:1090730007E007E007E007E007E007E007E007E0B5
:1090830007E007E007E007E007E007E007E0A637AF
:10909300B5F994F5A577B5F9ADD9ADD9ADD9ADD9B4
:1090A300ADD9ADD9ADD9ADD9ADD9ADD9ADD9ADF96D
:1090B300ADB8ADB73F8C07E007E007E007E007E096
:1090C30007E007E007E007E007E007E007E007E065
:1090D30007E007E007E007E007E007E007E007E055
:1090E30007E007E007E007E007E007E007E007E045
:1090F3005F4FBDDAA5B78CB4ADD8B5F9ADD9ADD94D
:10910300ADD9ADD9ADD9ADD9ADD9ADD9ADD9ADD92C
:10911300ADD9ADF9B5998E5407E007E007E007E054
:1091230007E007E007E007E007E007E007E007E004
:1091330007E007E007E007E007E007E007E007E0F4
:1091430007E007E007E007E007E007E007E007E0E4
:1091530007E007E08E95B5DAADD8A577B5F9ADD9B7
:10916300ADD9ADD9ADD9ADD9ADD9ADD9ADD9ADD9CC
:10917300ADD9ADD9ADD9ADD8B5785F2F07E007E04C
:1091830007E007E007E007E007E007E007E007E0A4
:1091930007E007E007E007E007E007E007E007E094
:1091A30007E007E007E007E007E007E007E007E084
:1091B30007E007E007E007E08E74B519ADB8ADF935
:1091C300ADD9ADD9ADD9ADD9ADD9ADD9ADD9ADD96C
:1091D300ADD9ADD9ADD9ADD9ADF9B5B99DD607E006
:1091E30007E007E007E007E007E007E007E007E044
:1091F30007E007E007E007E007E007E007E007E034
:1092030007E007E007E007E007E007E007E007E023
:1092130007E007E007E007E007E007E007E06EB1DB
:10922300A577AD38ADB8ADF9ADD9ADD9ADD9ADD917
:10923300ADD9ADD9ADD9ADD9ADD9ADD9ADF9B57933
:1092430076B207E007E007E007E007E007E007E0A2
:1092530007E007E007E007E007E007E007E007E0D3
:1092630007E007E007E007E007E007E007E007E0C3
:1092730007E007E007E007E007E007E007E007E0B3
:1092830007E007E037AC7672AD57AD38ADD8B5F926
:10929300B5D9ADD9ADD9ADD9ADD9ADD9ADF8ADF954
:1092A300ADD9AD983F8D07E007E007E007E007E0A1
:1092B30007E007E007E007E007E007E007E007E073
:1092C30007E007E007E007E007E007E007E007E063
:1092D30007E007E007E007E007E007E007E007E053
:1092E30007E007E007E007E007E007E0476D8E14BB
:1092F300AD37AD77ADD8B5F9ADD9ADD9ADD9ADD918
:10930300ADF8ADF9B599963507E007E007E007E05A
:1093130007E007E007E007E007E007E007E007E012
:1093230007E007E007E007E007E007E007E007E002
:1093330007E007E007E007E007E007E007E007E0F2
:1093430007E007E007E007E007E007E007E007E0E2
:1093530007E007E0574E9DD5AD37A598ADF9B5F9B0
:10936300ADD9ADD9ADF8ADF9B579673007E007E010
:1093730007E007E007E007E007E007E007E007E0B2
:1093830007E007E007E007E007E007E007E007E0A2
:1093930007E007E007E007E007E007E007E007E092
:1093A30007E007E007E007E007E007E007E007E082
:1093B30007E007E007E007E007E007E067119DB675
:1093C300AD38AD98ADF8B5F9ADF8ADB8A5D707E0B0
:1093D30007E007E007E007E007E007E007E007E052
:1093E30007E007E007E007E007E007E007E007E042
:1093F30007E007E007E007E007E007E007E007E032
:1094030007E007E007E007E007E007E007E007E021
:1094130007E007E007E007E007E007E007E007E011
:1094230007E007E07EB3A576AD38A5B8ADF8AD7813
:1094330076B207E007E007E007E007E007E007E0B0
:1094430007E007E007E007E007E007E007E007E0E1
:1094530007E007E007E007E007E007E007E007E0D1
:1094630007E007E007E007E007E007E007E007E0C1
:1094730007E007E007E007E007E007E007E007E0B1
:1094830007E007E007E007E007E037AB7692A57750
:10949300AD37AD77378C07E007E007E007E007E07B
:1094A30007E007E007E007E007E007E007E007E081
:1094B30007E007E007E007E007E007E007E007E071
:1094C30007E007E007E007E007E007E007E007E061
:1094D30007E007E007E007E007E007E007E007E051
:1094E30007E007E007E007E007E007E007E007E041
:1094F30007E03FAC7E92671007E007E007E007E074
:1095030007E007E007E007E007E007E007E007E020
:1095130007E007E007E007E007E007E007E007E010
:1095230007E007E007E007E007E007E007E007E000
:1095330007E007E007E007E007E007E007E007E0F0
:1097830007E007E007E007E0FFDFFFDFFFDFFFDFC2
:10979300FFDFFFDFFFDFFFDFFFDFFFDFFFDFF7BEFF
:1097A300FFDFFFDFFFDFFFDFFFDFFFDFFFDFFFDFC6
:1097B300FFDFFFDFFFDFFFDFFFDFFFDFFFDFFFDFB6
:1097C300FFDFFFDFFFDFFFDFFFDFFFDFFFDFFFDFA6
:1097D300FFDFFFDFFFDFFFDFFFDFFFDFFFDFF7BEBF
:1097E300F7DFF7DFF7DFF7BEF7BFF7BEF7BFF7BF68
:1097F300F7BEF7DFF7BEFFDFFFBEFFDFFFDFFFDFF1
:10980300FFDFFFDFFFDFFFDFFFDFFFDFFFDFFFDF65
:10981300FFDFFFDFF7BEF7BEF7BEF7BEF7BEF7BE4B
:10982300F7BFF7BEF7BEF7BEFFDFF7BEFFDFFFDF11
:10983300FFDFFFDFFFDFFFDFFFDFFFDFFFDFFFDF35
:10984300FFDFFFDFFFDFFFDFFFDFF7BEFFDFFFDF4E
:10985300FFDFFFDFFFDFFFDFFFDFFFDFF7BEFFDF3E
:10986300FFDFFFDFFFDFFFDFFFDFFFDFFFDFFFDF05
:10987300FFDFFFDFFFDFFFDFFFDFFFDFFFDFFFDFF5
:10988300FFDFFFDFFFDFFFDFFFDFFFDFFFDFFFDFE5
:10989300FFDFFFDFFFDFF7BEFFDFFFDFFFDFFFDFFE
:1098A300FFDFFFDFFFDFFFDFFFDFFFDFFFDFFFDFC5
:1098B300FFDFFFDFF7BEFFDFFFDFFFDFF7DFF7DFEE
:1098C300F7DEF7DFF7BEF7DFFFDFFFDFFFDFFFDFE7
:1098D300FFFFFFFFFFFFFFFFFFFFFFFFFFFFFFFF95
:1098E300FFFFFFFFFFFFFFFFFFDFF7DFF7DEEFDE27
:1098F300EFBEE7BEE7BEE7BEE7BFEFDEF7DFFFFF82
:10990300FFFFFFFFFFFFFFFFFFFFFFFFFFFFFFFF64
:10991300FFFFFFFFFFFFFFFFFFFFFFFFFFFFFFDF74
:10992300FFDFFFDFFFDFF7DFF7BEF7DFF7BEFFDFA6
:10993300FFDFFFDFFFDFFFDFFFDFFFDFFFDFFFDF34
:10994300FFDFF7BEFFDFFFDFFFDFFFFFFFDFFFDF2D
:10995300FFDFFFDFFFDFFFDFFFDFFFDFFFDFFFDF14
:10996300FFDFFFDFFFDFFFDFFFDFFFDFF7BEFFDF2D
:10997300FFDFFFDFF7BEFFDFFFDFFFDFFFDFFFDF1D
:10998300FFDFFFDFFFDFFFDFFFDFFFDFFFDFFFDFE4
:10999300FFDFFFDFFFDFFFDFFFDFFFDFFFDFFFDFD4
:1099A300FFDFF7BEF7DFF7DFFFDFFFDFFFFFFFFFBD
:1099B300FFFFFFFFFFFFFFFFFFFFF7DFDFBFCF7EED
:1099C300C73EAEDD9E7C9E1B8DDB6D5964F85CB893
:1099D3005C7754574C363C172B95237523351B3432
:1099E3001B351AF412F51AD31B141AF42314231477
:1099F3002B3433553B5543B64BB553B653F66498A6
:109A030085198D598DBAAE1BBE7CC6FDE77EF7BEA8
:109A1300FFFFFFFFFFFFFFFFFFFFFFFFFFFFFFDF73
:109A2300FFDFFFDFFFDFFFDFFFDFFFDFFFDFFFDF43
:109A3300FFDFFFDFFFDFFFDFFFDFFFDFF7BEFFDF5C
:109A4300FFDFFFDFFFDFFFDFFFDFFFDFFFDFFFDF23
:109A5300FFDFFFDFFFDFFFDFFFDFFFDFF7BEFFDF3C
:109A6300FFDFFFDFFFDFFFDFFFDFFFDFFFDFFFDF03
:109A7300FFDFF7BEFFDFFFDFF7BEFFDFFFDFFFDF45
:109A8300F7BEFFDFFFDFF7DFF7DFF7BFF7BFFFBF8C
:109A9300FFDFFFFFFFFFFFFFFFFFF7DFD79EC73D9E
:109AA300A6BC8E9C65FA65BA45792CD814570BD69B
:109AB30003B60355035502D4031502F402F402B4AA
:109AC300029302D4027302D4027302B402730253E8
:109AD300025301F2021201B1021201F202530A739C
:109AE30012931AB41AF42375335543754B75539572
:109AF3004BB543954395439543B53BD643B753B6CF
:109B03006CB864B86D398E3BAE9CC71DDF5EEFBF8A
:109B1300FFBEFFDFFFDFFFDFFFDFFFDFFFDFFFDF73
:109B2300FFDFFFDFFFDFFFDFFFDFFFDFF7BEFFDF6B
:109B3300FFDFFFDFFFDFFFDFFFDFFFDFFFDFFFDF32
:109B4300FFDFFFDFFFDFFFDFFFDFFFDFFFDFFFDF22
:109B5300FFDFFFDFFFDFFFDFFFDFFFDFFFDFFFDF12
:109B6300FFDFFFDFFFDFFFDFFFDFFFDFFFDFFFDF02
:109B7300F7DFF7DFFFDFFFDFFFFFFFFFFFFFFFFF82
:109B8300DF9EB71D8E9C5DDA45993D592D39457A87
:109B93003D79359A24F80CF90457041703F603D6D4
:109BA30003F703950417039503B60375037503952C
:109BB3000375037502D40315029302D40AF41355F3
:109BC3002BD65C576CF98DBA9E3CBEBDD71EE7BF42
:109BD300EFDFF7DFFFFFFFFFFFFFFFFFFFFFFFFFEA
:109BE300FFFFFFFFFFFFFFFFFFFFFFFFF7DFEF7E3B
:109BF300E75ECEFDBE9CAEBC965B9E9C965BA6BC10
:109C0300BEBCDF3EF7BEFFDFFFDFFFDFFFDFFFDFAF
:109C1300FFDFFFDFFFDFFFDFFFDFFFDFFFDFFFDF51
:109C2300FFDFFFDFFFDFFFDFFFDFFFDFFFDFFFDF41
:109C3300FFDFFFDFFFDFFFDFFFDFFFDFFFDFFFDF31
:109C4300FFDFFFDFFFDFFFDFFFDFFFDFFFDFFFDF21
:109C5300FFDFFFDFFFDFF7BEF7BEF7DFF7DFFFFF53
:109C6300FFFFFFFFFFFFEFDFB71D865C5DDB3519ED
:109C73001D3A351955DB7E5C9EFDCF7EEFBEEFFFAF
:109C83006E5B2D190417041703D604170437041643
:109C9300043703D6041703B603F603B50376035557
:109CA30002D403761BB644B96D799E5BC71DE7BE2C
:109CB300FFFFFFFFFFFFFFFFFFFFFFFFFFFFFFDFD1
:109CC300FFDFFFDFFFBEFFBFFFBFF7BFF7BEF7BE7C
:109CD300F7BFF7BEF7BFFFDFFFDFFFDFFFDFFFDF0A
:109CE300FFFFFFFFFFFFFFFFFFFFFFFFFFFFF7DFA9
:109CF300F7BEF7BEF7BFFFDFFFDEFFDFFFDFFFDFEC
:109D0300FFDFFFDFFFDFFFDFFFDFFFDFF7BEFFDF89
:109D1300FFDFFFDFFFDFFFDFFFDFFFDFFFDFFFDF50
:109D2300FFDFFFDFFFDFFFDFFFDFFFDFFFDFFFDF40
:109D3300FFDFFFDFFFDFFFDFFFDFFFDFFFDFFFDF30
:109D4300FFDFFFDFFFDFFFDFFFDFFFFFFFFFE7BF18
:109D5300B6FD765B3D79151925193D7A7E3CB6FD36
:109D6300DF9EF7DFFFFFFFFFFFFFFFFFFFDFFFDFE9
:109D7300F7DFEFBEC75D8E9C457A24B8043703D660
:109D830003F703D60457039603B603B61C374519E6
:109D93008DFBC73EEFBEFFFFFFFFFFFFFFFFFFDFB0
:109DA300FFDFF7BEF7BFF7BEF7DFF7BFFFDFFFDF6A
:109DB300FFDFFFDFF7BEFFDFFFDFFFDFFFDFFFDFD9
:109DC300FFDFFFDFFFDFFFDFFFDFFFDFFFDFF7BFC8
:109DD300FFDFFFDFF7BFF7BFF7BEF7DFFFDFFFDF11
:109DE300FFDFFFDFFFDFFFDFFFDFFFDFFFDFFFDF80
:109DF300FFDFF7BEFFDFFFDFFFDFFFDFFFDFFFDF99
:109E0300FFDFFFDFFFDFFFDFFFDFFFDFFFDFFFDF5F
:109E1300FFDFFFDFFFDFFFDFFFDFFFDFF7DFFFDF57
:109E2300FFDFFFDFFFDFF7DEFFDFFFDFFFDFFFBE69
:109E3300FFDFFFDFFFDFFFDFD79E7EDC3DBA2519A3
:109E43001CB83D9A7E5BBF3DEFBFFFFFFFFFFFFFE7
:109E5300FFDFF7BEF7BFF7DFF7DFF7BEFFDFFFDF99
:109E6300FFDFFFDFFFFFFFFFFFFFE7BEC73D8E5BA7
:109E73004D5A1C770C58247875DBB6FDE79EFFFF1F
:109E8300FFFFFFFFFFDFF7BEF7BEF7DFFFDFF7DF01
:109E9300FFDFFFDFFFDFFFDFFFDFF7BEFFDFFFDFF8
:109EA300FFDFFFDFFFDFFFDFFFDFFFDFFFDFFFDFBF
:109EB300FFDFFFDFFFDFF7BEFFDFFFDFFFDFF7BE01
:109EC300FFDFFFDFFFDFFFDFFFDFFFDFFFDFFFDF9F
:109ED300FFBFFFBFFFDFFFDFFFDFFFDFFFDFFFDFCF
:109EE300FFDFF7BEFFDFFFDFFFDFFFDFFFDFFFDFA8
:109EF300FFDFFFDFFFDFFFDFFFDFFFDFFFDFFFDF6F
:109F0300FFDFFFDFFFDFFFDFF7DFF7DFFFDFFFDF6E
:109F1300F7BEF7BEF7BEF7BEF7BEF7BEFFDFFFDF44
:109F2300FFDFF7BEF7BEFFBEC73D8EDC96BCBF1D8D
:109F3300E7BEFFFFFFFFFFFFFFBEFFBEF7BEF7BF9A
:109F4300FFDFF7DFFFDFFFFFFFDFFFDFF7BEFFBE50
:109F5300FFDFF7DFF7BEF7BEF7BEFFBEFFDFFFFF92
:109F6300FFFFE79ECF5DF7FFFFFFFFFFFFDFF7BEBA
:109F7300F7DFF7BEF7BEF7BEF7BEF7BEFFDFF7BEEC
:109F8300F7BEF7BEF7BEF7BEF7BEF7BEF7BEF7BE26
:109F9300FFDFFFDFF7BEF7BEF7BEF7BEF7BEF7BEC4
:109FA300F7BEF7BEF7BEF7BEF7BEF7BEF7BEFFDFDD
:109FB300FFDFFFDFFFDFFFDFF7BEF7BEF7BEFFDF29
:109FC300F7BEFFDFFFDFFFFFFFFFFFDFFFDFFFDF87
:109FD300FFDFFFDFFFDFF7BEF7BEF7BEF7BEF7BE5B
:109FE300F7BEF7BEFFDFF7BEFFDFF7BEF7BEF7BE74
:109FF300FFDFFFDFFFDFFFDFFFDFFFDFFFDFFFDF6E
:10A00300FFFFFFFFFFFFFFFFFFFFFFFFFFDFF7BEC6
:10A01300F7BEFFFFFFFFFFFFFFFFFFFFFFFFFFFF96
:10A02300FFFFF7BEF7DFF7FFFFFFFFFFFFFFFFFFB6
:10A03300FFFFFFDFFFBEFFBEFF9EFFDFFFFFFFFF50
:10A04300FFDFFFFFFFFFFFFFFFFFFFFFFFFFF7DF65
:10A05300F7DFFFFFFFFFFFDFF7DFFFFFFFFFFFFF7D
:10A06300FFDFFFFFFFFFFFFFFFFFFFFFFFFFFFFF1D
:10A07300FFFFFFFFFFFFFFFFFFFFFFFFFFFFFFFFED
:10A08300FFDFFFFFFFFFFFFFFFFFFFFFFFFFFFFFFD
:10A09300FFFFFFFFFFFFFFFFFFFFFFFFFFFFFFDFED
:10A0A300FFDFFFDFF7BEFFFFFFFFFFFFFFFFFFFF46
:10A0B300FFFFFFFFF7BEF79EF79EF7BEFFDFFFFF31
:10A0C300FFFFFFDFFFDFFFFFFFFFFFFFFFFFFFFFDD
:10A0D300FFFFFFFFFFFFFFFFFFFFFFFFFFFFFFFF8D
:10A0E300FFDFFFDFFFDFFFDFFFDFFFDFF7BEFFDFA6
:10A0F3008430630C632C632C738EAD55F79EFFFF86
:10A10300FFFFD69A8410630C630C5B0C634DDEFB7C
:10A11300FFDFFFFFFFFFFE59FCB2FB4DFACBF9C790
:10A12300F924F924F9A6FA08FA49FA69FA69FAEB63
:10A13300FF1CE75D6B6D630C630C630C9CF3FFFF0B
:10A14300FFDFFFDFFFDFFFDFFFFFAD75630C9CD396
:10A15300FFFFDEDB632C630C630C630C5AEB528A48
:10A163004A694A69528A4A69528A528A528AB59618
:10A17300FFDFEF5D6B6D630C630C630C5AEB528A6C
:10A18300528A528A528A528A5ACB8410B5B6FFDF5A
:10A19300FFDFFFDFFFFFE73CB5968410630C4A69DE
:10A1A30031862124296542084A49528A528A528AB1
:10A1B3009492FFDFFFFFBDF78C516B4D630C52AAE6
:10A1C3004A694A494A494A494A69528A7BEFD69AB7
:10A1D300FFFFFFDFFFDFFFDFFFDFFFDFF7BEFFFF75
:10A1E30031860000000000000000000029658C514A
:10A1F3005ACB000000000000000000000000AD5535
:10A20300FFFFF659F9E7F841F800F800F800FAAA59
:10A21300FD14FE59FEBAFEFBFF1CFEBAFE59FE18E2
:10A22300FFBEBDF7000000000000000031A6FFFFE5
:10A23300F7BEFFDFFFDFF7BEFFFF4A4900003186AD
:10A24300FFFFB596000000000000000010A2AD550E
:10A25300B5B6B5B6B5B6BDD7B5B6B5B6B5B6DEDB2C
:10A26300FFFFC618000000000000000010A29CD3EE
:10A27300A534A534A534A5148C71210400006B6D9D
:10A28300FFFFFFDF7BEF18C300000000000010A2F8
:10A293008410BDD7D6BAEF7DF79EEF7DDEFBCE7976
:10A2A300D6BAFFFF7BCF00000000000000006B6DFB
:10A2B300B596BDD7BDD7B5B6B5B67BEF000008617F
:10A2C300D69AFFDFF7BEFFDFFFDFFFDFF7BEFFFF3B
:10A2D30042080000630C632C0841000000000000EA
:10A2E3000841843042080000002000200000B5B679
:10A2F300FF7DF0E3F800F800F820F800FC51FFFFC1
:10A30300FFFFFFFFFFFFFFFFFFFFFFFFFFFFF7FF62
:10A31300FFFFBDF700000020002000004208FFFF00
:10A32300F7BEFFDFFFDFF7BEFFFF528A00004208E0
:10A33300FFFFBDD7000000200020000018E394B207
:10A343009CF39CF39CF39CF39CF39CF3CE59FFFF8B
:10A35300FFFFC63800000020002000004228FFFF56
:10A36300FFFFFFFFFFFFFFFFFFFF8C5100002945A9
:10A37300FFFF8C71000000000020002018E3E71CA1
:10A38300FFFFFFFFEF7DD69AD69AD69ADEFBE73C16
:10A39300FFDFFFFF31A60000002000200000738EC6
:10A3A300949294929492949294927BCF0020000082
:10A3B300B5B6FFFFF7BEFFDFFFDFFFDFF7BEFFFF2F
:10A3C30042080000AD55FFFFCE7994926B6D94B2B5
:10A3D300E71CFFFF5AEB0000000000000000B5F788
:10A3E300FE9AF000F820F800F800F800FE79FFFF6D
:10A3F300FF9EFFBEFFBEFFBEFFBEFFBEFFBEF79EBA
:10A40300FFFFBDF700000020000000004208FFDF4F
:10A41300F79EF7BEF7BEF79EFFDF528A000039E7CB
:10A42300FFFFBDD7000000000000000000204A69C4
:10A433005ACB5ACB5ACB5ACB5ACB5ACB8410FFDFC9
:10A44300FFFFC6380000000000000000084152AAC8
:10A45300632C630C630C5AEB4A6908412965A534E4
:10A46300FFFF422800000020002000004228FFFFD9
:10A47300F79EF7BE843039C739C7318608610000BB
:10A483004A69FFFF42080000000000000000420884
:10A49300738E738E738E738E738E4A490000000021
:10A4A300BDF7FFFFFFDFFFDFFFDFFFDFF7BEFFFFCC
:10A4B300420800009CD3FFDFFFFFFFFFFFFFFFFF0A
:10A4C300FFFFFFDF528A0000002000200000B57567
:10A4D300FFDFFA69F800F800F800F800FA8AFF3C99
:10A4E300FFFFFFFFFFFFFFFFFFFFFFFFFFFFF7FF81
:10A4F300FFFFBDF700000000000000004208FFFF5F
:10A50300FFFFFFFFFFFFFFFFFFFF528A000039E756
:10A51300FFFFBDD7000000000000000039C7FFFFA8
:10A52300FFFFFFFFFFFFFFFFFFFFFFFFFFFFF7BE81
:10A53300FFFFCE59000000000000000018E38C511B
:10A543008C718C518C518C71A534CE79F79EFFFFA1
:10A55300FFFFBDF700200000000000001082BDF7E0
:10A56300FFFFFFFFFFFFFFFFFFFFFFFF5ACB0000CF
:10A5730039C7FFFF39E70000002000200000CE5953
:10A58300FFFFFFFFFFFFFFFFFFFFD6BA0000000042
:10A59300BDF7FFFFF7BEFFDFFFDFFFDFF7BEFFFF04
:10A5A300318600009CF3FFFFF7BEF7BEF7BEF7BE90
:10A5B300F7BEFFFF52AA0000000000000000B5B67E
:10A5C300FFFFF79EFC51F986F882F800F800F84186
:10A5D300FA28FBCFFC92FC92FC92FC71FC51FC101C
:10A5E300FF1CEF7D630C10A2002000000000420856
:10A5F3005ACB5AEB5AEB5AEB42280000000039E7DA
:10A60300FFFFEF7D738E21040841000031A6FFDFB9
:10A61300F7BEF7BEF7BEF7BEF7BEF7BEF7BEFFDF66
:10A62300FFDFF7BE738E18C30000000039E7FFFF9A
:10A63300FFFFFFFFFFFFFFFFFFFFFFFFFFDFF7BE90
:10A64300FFDFFFFFC6385ACB18E3084100000000C4
:10A653004A698C7194B294B294928C511082000026
:10A6630031A6FFFF39C70000000000000000BDD77E
:10A67300FFDFF79EF7BEF79EFFDFC638000000003E
:10A68300BDD7FFFFFFDFFFDFFFDFFFDFFFDFFFDF01
:10A69300BDD7A534EF7DFFDFFFDFFFDFFFDFFFDF88
:10A6A300FFDFFFDFDEDB9CF39CF39CF3AD55F79EEE
:10A6B300FFDFFFDFFFFFFFDFFEBAFDD7FCF3FC5137
:10A6C300FB4DFAEBFAEBFAEBFB0CFBAEFC30FCD3E5
:10A6D300FF7DFFFFFFFFDEFBC618A5349CF38C71E3
:10A6E3008C718C718C718C718C719CF3A534D69A9E
:10A6F300FFDFFFDFFFFFEF5DCE59AD75CE79FFDFE3
:10A70300FFDFFFDFFFDFFFDFFFDFFFDFFFDFFFDF56
:10A71300FFDFFFDFFFFFE71CBDF79CF3D69AF7BE11
:10A72300F7BEF7BEF7BEF7BEFFDFF7BEFFDFFFDF03
:10A73300FFDFFFDFFFFFFFFFEF5DC638AD559CD3A3
:10A7430073AE630C5ACB5ACB5AEB6B4D84309CD30C
:10A75300CE59FFDFCE79A5149CF39CF3AD75F79E1C
:10A76300FFDFFFDFFFDFFFDFFFDFF7BEB596AD558E
:10A77300EF7DFFDFFFDFFFDFFFDFFFDFFFDFFFDF58
:10A78300FFFFFFFFFFFFFFDFFFDFFFDFFFDFFFDF76
:10A79300FFDFFFDFFFFFFFFFFFFFFFFFFFFFFFFF06
:10A7A300FFDFFFDFFFBEFFDFFFFFFFFFFFFFFFFF57
:10A7B300FFFFFFFFFFFFFFFFFFFFFFFFFFFFFFFFA6
:10A7C300FFFFFFDFF7BEFFFFFFFFFFFFFFFFFFFFFF
:10A7D300FFFFFFFFFFFFFFFFFFFFFFFFFFFFFFFF86
:10A7E300FFDFFFDFF7BEFFFFFFFFFFFFFFFFFFDF1F
:10A7F300FFDFFFDFFFDFFFDFFFDFFFDFFFFFFFDF46
:10A80300FFDFFFDFF7BEFFFFFFFFFFFFFFFFFFDFFE
:10A81300FFDFFFDFFFDFFFFFFFFFFFDFFFDFFFDF05
:10A82300FFDFFFDFFFDFFFDFFFFFFFFFFFFFFFFFB5
:10A83300FFFFFFFFFFFFFFFFFFFFFFFFFFFFFFFF25
:10A84300FFFFFFDFFFFFFFFFFFFFFFFFFFFFFFFF35
:10A85300FFDFFFDFFFDFFFDFFFDFFFDFFFFFFFFFC5
:10A86300FFFFFFDFFFDFFFDFFFDFFFDFFFDFFFDFD5
:10A87300F7BEF7BEFFDFFFDFFFDFFFDFFFDFFFDF37
:10A88300FFDFFFDFFFDFF7BEF7BEF7BEF7BEFFDF79
:10A89300FFDFFFDFFFDFFFDFFFDFFFBEFFBEFFBE28
:10A8A300FFBEFFBEFFBEFFBEFFBEFFBEFFBEFFBEBD
:10A8B300FFDFFFDFFFDFFFDFF7BEF7BEF7BEF7BE49
:10A8C300F7BEF7BEF7BEF7BEF7BEF7BEF7BEFFDFB4
:10A8D300FFDFFFDFFFDFFFDFFFDFF7BEF7BEFFDFD7
:10A8E300FFDFFFDFFFDFFFDFFFDFFFDFFFDFFFDF75
:10A8F300FFDFFFDFFFDFFFDFFFDFF7BEF7BEFFDFB7
:10A90300FFDFFFDFFFDFFFDFFFDFFFDFFFDFFFDF54
:10A91300FFDFFFDFFFDFFFDFFFDFFFDFF7BEF7BE96
:10A92300F7BEF7BEF7BEFFDFF7BEF7BEF7BEF7BE53
:10A93300FFDFFFDFFFDFF7BEF7BEF7BEF7BEFFDFC8
:10A94300FFDFFFDFFFDFFFDFFFDFFFDFF7BEF7BE66
:10A95300FFDFFFDFFFDFFFDFFFDFFFDFFFDFFFDF04
:10A96300FFDFFFDFFFDFFFDFFFDFFFDFFFDFFFDFF4
:10A97300FFDFFFDFFFDFFFDFFFDFFFDFFFDFFFDFE4
:10A98300FFDFFFDFFFDFFFDFFFDFFFDFFFDFFFDFD4
:10A99300FFDFFFDFFFDFFFFFFFDFFFDFFFDFFFDFA4
:10A9A300FFDFFFDFFFDFFFDFFFDFFFDFFFDFFFDFB4
:10A9B300FFDFFFDFFFDFFFDFFFDFFFDFFFDFFFDFA4
:10A9C300FFDFFFDFFFDFFFDFFFDFFFDFFFFFFFDF74
:10A9D300FFDFFFDFFFDFFFDFFFDFFFDFFFDFFFDF84
:10A9E300FFDFFFDFFFDFFFDFFFDFFFDFFFDFFFDF74
:10A9F300FFDFFFDFFFDFFFDFFFDFFFDFFFDFFFDF64
:10AA0300FFDFFFDFFFDFFFDFFFDFFFDFFFDFFFFF33
:10AA1300FFDFFFDFFFDFFFDFFFDFFFDFFFDFFFDF43
:10AA2300FFDFFFDFFFDFFFDFFFDFFFDFFFDFFFDF33
:10AA3300FFDFFFDFFFDFFFDFFFDFFFDFFFDFFFDF23
:10AA4300FFDFFFDFFFFFFFDFBD59A474E679E69761
:10AA5300D5D2EE95E635E5F5EE57FED8EE75EE74F4
:10AA6300FF17F6D7ACD1A470B4F2B512A4B0942EEC
:10AA7300ACD1A470A491A4719C91A492ACD3A4B3BF
:10AA8300A493A4B3ACF5A4B4A4B5A4D6ACF69C9497
:10AA9300949394D48C928C937C527C737433849669
:10AAA30084D88CD974379D5B95178CD595168CF506
:10AAB3008CD5951694D68CB594B69CF79CB79CD739
:10AAC300ACB7CD99D6176AA76265EE95DDF46A2611
:10AAD3008B2AE5F5EE34B4CEC530E6969C0E49A537
:10AAE300ACB0BD526AC949C583ADB5137B4C5A2876
:10AAF3006AEB9430BD76BD75BD55ACF4B515B5158F
:10AB0300BD57ACF6A4B49CD48C3173CF843184711B
:10AB13007411743284B4745484B77C768CD9953AA6
:10AB2300849574127C73741273D16BD17BF37C3371
:10AB3300A538AD59A518AD39ACD8B4F6E679CDB37F
:10AB4300C571FEF6D5928B2A9BCCE635EE75C550C2
:10AB5300CD71EE96AC9072C99C2FC573940E6AC9E1
:10AB63007B6C9C707B4B6ACA838D8BCE8BCF7B6D4A
:10AB73008C109C519C718BF09431943294517BAE28
:10AB830083EF84506B6D73EE73EF74107C9384D5F5
:10AB93008D177C7584B87C9684954ACD42AC4AED7A
:10ABA3005B2F428C4A6D52EE8C559CF794969CB663
:10ABB300C57AACB6DE38E697DE34F6B5F696FEB85F
:10ABC300EE36F676EE54EE74EE95E675BD12BD5391
:10ABD300B512B512B5328BCD940EACF1ACF283AD98
:10ABE300942FACF2BD74B5549450B534CDD6C5D6BC
:10ABF300A492A4D3734C6B2BA512B594AD94CEB889
:10AC0300A5948CD25B6D7C7284D584B57C969D793A
:10AC130063D1532E4AED42AC4AAD63705AEF4A6D8D
:10AC23008414AD79AD59AD39ACB7B4D6DE58E697D7
:10AC3300E654FEF6F696E615F677EE56EE54F6B5BE
:10AC4300F6D6E696BD12BD33BD53A4B09C4F72EA4F
:10AC5300940EC5B4C59483ADACF1C5D5CE16CDF66F
:10AC63006B0A9470AD12ACF2E6B9CE1683CDB55330
:10AC7300C615948EB5B3C656E75ACED984907C5187
:10AC83008CF484B46BF295583A4B3A4B3A6C530EAE
:10AC93003A4C52EE426C52EF52AE94969CD7949635
:10ACA300C57ABD17DE38F719F6D6EE95EE56F69748
:10ACB300F657F677F695F6D6F6D6EED7BD32A491CB
:10ACC300B533A4907B6B838CB512CDD5942EA49011
:10ACD300CE15C5B4944E944E6B0ABDB4BDB4A4F165
:10ACE300A4B07B8BBD73CE35AD30B572BDB3BDF3B0
:10ACF300AD93C656B5F57C50955595358CD5A5B90C
:10AD03004ACD3A6B428C63904ACE530F4A6D5B3007
:10AD130063309CF7B579AD38ACB7B4F7DE58EED8ED
:10AD2300EE95EE74EE56F677F697F676F675F6D65A
:10AD3300EEB5EE96BD12A470BD538BCD6AEAACF1AD
:10AD4300EED9CDD5734BB512E6B8E6D8A4D08C2D89
:10AD53009CAFD676B572948E8C0D83CCEF19A4CFAD
:10AD63007349C5F3AD30A530AD92BE35CED97C5015
:10AD73006BF07C737C738D16534F532F530E322B12
:10AD8300426C639163303A2C739294969CD79CD710
:10AD9300BD19BD58D617E697EE95F6B5F696F65754
:10ADA300EE57F697FEB6FEF6EEB5EEB6BD129C5024
:10ADB300A4706AC98BCDB512D6369C8F7B8BBD73BD
:10ADC300D635DEB7944D62E8B592DE96A510944D64
:10ADD3006AE8B532C5B383AB62E783CB7B8A5AC7D4
:10ADE300840C8C6FBE169D1363AF953684B4953770
:10ADF30084B54ACE530F4ACE6B914ACE635073D378
:10AE03009CF8A538A519AD59ACD8B4F7DE58F6F8B7
:10AE1300F6D6F6B5F676FE98F697F697F6B6F6B545
:10AE2300EEB5F6D7B4F1A470940E5A885A47B553C9
:10AE3300DE978BCD6AE9C5D4E6F8D6557BCB4A2499
:10AE43006B49C613B5927BAA5246CDD5DE97ACF0BB
:10AE5300734983CB7B8A5AA752875AE98C71ADB663
:10AE63006BD07C538CF684B66BF3530F42AE4ACE51
:10AE73005B304ACE4A8E73B2841494B6A518A4F8F4
:10AE8300ACD8B4F7DE38EED8EEB6F6B5EE76F69774
:10AE9300F697F677F6B6F6B5EEB5F6D7B512A490F3
:10AEA300942F52267B8C9C6FCDF58BED5226AD51A2
:10AEB300DED7CE357BAB62E79CAEB591E6F7A4EF68
:10AEC3005A8783ACCDF5E6B8B531B531B5318C2DA4
:10AED3005AC85AEA8C51A555638F8CF6849584B66B
:10AEE3006BD25B715B504ACE52CE530F5B1073B281
:10AEF3007BD39496A4F89CD8B4F8B517DE38EED774
:10AF0300EEB5F6B5EE76F697F697F677F6B6F6B5AE
:10AF1300EE95F6D7B4F1A4908BCD8BED83CD8C0E4B
:10AF2300C5B4AD118C0D840CB551E6D7AD519CAEB3
:10AF330073AAA530DED6BDB3946F83CDA4D0C5D498
:10AF4300E6D8CE15A4AFA4D0840E73ADA5559D1538
:10AF530074129D58745574344B0F533063B253308D
:10AF630052EF6BB26B714A8E63318435A4F8A51826
:10AF7300B518BD17DE58EED8EEB6F6B5F676FE98E0
:10AF8300FE98F697F6B6F6B5EE95EEB7B4D19C4FAC
:10AF93007B4BBD5383CCACF1C5D4C5D4B5527BAB8D
:10AFA300D656E6F7B592AD307BCBDEB7CE349CCF29
:10AFB300A5116B2AAD32D636E6B7DE97B57283EDAF
:10AFC30083EE73ADAD7573F0849484D67C9563D3AF
:10AFD3004AEF530F63924AAE320C635173D35AF064
:10AFE300528E73929CB7A518B519BD17DE38EED8EB
:10AFF300EEB6F6B5F676FE98F697F697FEB6F6B584
:10B00300EEB5EEB6ACB09C2F7B4B9C8F946FBDB46A
:10B01300BDB4A4F08C2E8C2DDED8AD51840C83EB03
:10B023009CAECE35B5B373AB8C2D738BC5F4CE35D7
:10B03300C5F4CDF4B572944E949094B1A555634E76
:10B04300849474337C9663D363926BD284966BB38C
:10B05300426E637284557BF46B518435A518AD59E8
:10B06300B4F8BD17DE38EED7EEB6F6B5F676F6973A
:10B07300F677F677F6B6F6B5EEB5EED7B4D19C2FE4
:10B08300734B8C0D9C8FAD11CE358C2D9C8F8C0DFD
:10B09300CE35D676948F9CCF9CD0BDD3D6979CD0FB
:10B0A3008C2D94AFBDD3BDB3CE14C5D3AD11B57242
:10B0B300B593C616A5556BAF7C937C9484F784D661
:10B0C3007C756BD384767C556B927C1484356B9240
:10B0D30084148C769CD79CD7B4F8B517DE38EED899
:10B0E300F6D6F6D6F676F697F677F677F6B6F6B59B
:10B0F300EEB5F6D7B4F1A47083AC8BED9C8F9C6F47
:10B10300D656A4D0B572946EAD32DED8A4D0A4F0D6
:10B113008C4EBDD4CE769CF094AF842CAD71DEB64C
:10B12300D655DED6DED7BDB3AD52B5B49D335B4D38
:10B1330084B38D3685169DBA8D1863B25B51531057
:10B1430052F06BB373D36B72A539AD59AD39AD39C9
:10B15300B4F8B517DE38EED8F6F7F6F7F696F6B785
:10B16300F6B8F697F6B6EE96EEB6F6D7BD12ACB0D5
:10B173009C6F6B09B5729C8FBD93BDB38C4EBDB3F1
:10B183009CAFB572C5F49CD0A4F0A4F0B572AD72B7
:10B1930094AFA53094AEAD30B591CE34CE14CE3548
:10B1A300BDF5B5D5B5F7532C8D158CF56C538517B7
:10B1B3008CD774147C346BB35B316B927C148C76B8
:10B1C3009496949694979CB7BD38B4D6DE59E67896
:10B1D300DE56E675F6F8F6D7E676EEB7FF39EE9764
:10B1E300F6D8EEB7BD32A48F9C8F63099CD0948FA1
:10B1F3006309A5118C2DAD318C4E83ECBDD3944ED8
:10B20300A4F06B49840CA4F083EC9CAE7369944D59
:10B21300A4CFC5F4C635CE77CE78B5F6BE386BAFBE
:10B22300741184D595378D179538951895188CB763
:10B233008C969D18A539B59AA518A4F8B57AB55971
:10B24300B4D6BD16EE9BBD3462A8940CE696EEB65A
:10B25300F718EEB7ACD0ACB08B8BD5D4BD11ACAF77
:10B26300AD11736B4A465266736BAD32C5D48C2DE8
:10B273005246A510CE55A4F083EC4A25946ECE35E4
:10B28300ACF052457B8AA4CFBDD3B573CE77B5D589
:10B29300C6378C91849273F0951584B47C747C5476
:10B2A300741374137C3473F373F3843473B26B5178
:10B2B3007BB37B9294559CB6B4B5B4B4E65AD5F639
:10B2C300940DB4F0E696E655EE96DE148B8BAC6FD8
:10B2D3007B09DE15C5529C4EA4B09CB0736B8C2EBB
:10B2E300A4F1B552DE98B573B552A4D0AD31E6B82A
:10B2F300C5D4A4AFB552B531CE35A4CF946E9C8FCF
:10B30300A4F0B5939CB09D127BEE73CE73EF52EC19
:10B313005B4E6BB08CB495167C548D179D387413AB
:10B3230073F39CF7A5189CB69CD79455A4D7AD3955
:10B33300CD78C536CD97A4709C2D9C0CC571EED6E7
:10B34300EE96E656A44EAC8F9BEDC552C552AC8F1C
:10B35300BD738C2E734BC5B4D657D636A4D1AD125C
:10B36300DE77B532BD93B5539C6FBD93BD73A4B067
:10B373009C6FA4D0D656AD11946E8C4E8C4F5AE967
:10B383005AEA3A0729A63208424A29C83A4A4AAD34
:10B39300639074548CD68475845494D68434739295
:10B3A3009CB68C35A4B7AD18AC95BD36EE9BCDB627
:10B3B300EEB8D614E696EED7E696F6F8CD93CD73AF
:10B3C300CD93C552BD11BD11ACF183CD944FCDF6D4
:10B3D300AD128BEE6AEAC5B4C5D5B5338BCD62A980
:10B3E300A4D1CDF69C7083CD736BB553C5F5AD3247
:10B3F300736B4226420539C53A0652A94A693A088F
:10B40300298631C83A2A3209322A196729C9530EC3
:10B41300845494B57BF37BD37BB27BB29C96A4F824
:10B42300BD17ACB5E67AE658E677ACCFACAF942C53
:10B43300A48EBD119C0DC552EEB8EE97B4D0ACD01E
:10B44300ACF2942F942FA4B19C70732B734CACF279
:10B453009C70A4B17B8D7BADB5339C90945083CD10
:10B46300736CCE168C0E7BCD52884A674A479490F4
:10B473006B6C3A0729645AEB5AEC4A8B3A095B0D19
:10B483007432532E3A4B31EA5B0E8C959CD69CD684
:10B49300A4D79CB6B539B539B517ACD6D619E69A43
:10B4A300CDD59C4E942DACD09C8E9C4E8BACACB128
:10B4B300D616E6B8B512B4F1AD12A4D19CB19CB1C5
:10B4C3009C91945094709CB1A4F2AD13A4D2947146
:10B4D3009471A4F3C5F78C509C919CB19CD26B4C96
:10B4E300528842277BEE8C4F738D6B4C6B6D84506F
:10B4F30073AE7BEF4A6A52CC5B6F5B8F4AED29C90F
:10B50300426C8C749CF794B69CD79455A4B7A4F85A
:10B51300ACF8ACF77B90732D8BEE9CB0736B8C2DDA
:10B5230083ED8BED9C908BCE83AD7B6C62A962C95E
:10B533006B0A62EA6B2B630A4A27738C528962EBAC
:10B543006B2B52A96B4C738D6B6D6B6D5AEB738DBB
:10B55300738D6B2C736D5AEA52895289632B9D123A
:10B563008C505AEA42275B0B6B6E94B3528A424A61
:10B573005B4E3A8B320929E94A8C6B706B7073719D
:10B5830062EF5AAF83F4AD189CB79CB76B4F62CC94
:10B59300632B52A95AC96B2A630A5A886B2B5A899F
:10B5A30052284A075A6852474A274A4742274A6855
:10B5B3004A884A684A68420739E739E742485AEBFA
:10B5C3005B0C4AAA4A6A52AA630C526931A639E74C
:10B5D3005ACA52AA52CA7BCE73AD422842284A693C
:10B5E3004A694A6A422952EC5B4E4B0D4ACC428C63
:10B5F300424B3A0A420B422C5ACF526D7B92A4D84B
:10B60300B57AAD397BB1630D630C4A684226424774
:10B6130052884206528942084A2852695ACA5AC96C
:10B623004A474A684A6852A952C952A94A894228D4
:10B6330042083A0842695AEC5B0C52CB4AAB52CCF3
:10B643006B6E62EC4A2939E84A494A4942284A89D9
:10B653005B0B4AAA4AAA3A2831E8426A424A426A3A
:10B663003A4B322A322A320A3A0A39EA39EA420B87
:10B673005AAF5A8E83D4B5399CD894966B2F5AAC53
:10B683005ACB4A684A474A6752A94A2752894A48C5
:10B6930052695AAA5AA9526852A8528852885288A3
:10B6A30052A952A952894A694A4942494A8A5AECDB
:10B6B30052EC52AB4AAB52CC52AC528B4A4A39E8A9
:10B6C30042294A8A4A8A424942694A8A4AAB3A0823
:10B6D30031E8426A426A426B3A4B324B322B3A4B65
:10B6E3003A2C3A0B420B420C4A2D4A2D7372A4B8E2
:10B6F300AD39B559A4F6AD15B595B594B573BDB4CB
:10B70300BDB4B553BD95B574B575B5549C918C0E48
:10B713009C908C2E8C0E83CD83EE8C2F8C2F8C5192
:10B72300843084318C518C728C52843184328452B3
:10B733008C528C538C327BF173D07C317C106BAE8A
:10B74300636D5B4D636E63AF6BAF638F63B07C53AD
:10B753007C747C747C547C548454841484148414C6
:10B7630083D37BB39456AD19ACD7B558CE1ADE9AB2
:10B77300EEFAE6D9DE97DEB7DEB7DE97E698E6990E
:10B78300E6B9E698BD53A4B1B5129C6F9C70940FB3
:10B79300942F9C719C51A4D39CB2A4B3A4B39CB426
:10B7A3009C9394939C949CB49CD59CD59CD59CD4FD
:10B7B3008C738C7384727C117C527C31743184D48D
:10B7C300953684B484D49D988CD684B68CB68CB6C6
:10B7D30094B794B79CD7A4F8A4D79CB7A4B8A4F8FB
:10B7E300B4F7BD37D63ADE9ADE98DE97DE56E69694
:10B7F300DE76DE77DE57DE57E678E677BD32ACD10C
:10B80300BD12A46FACB1A470A491ACB29C50A4B30C
:10B81300A4B3ACD4ACF4A4D4A4B4A4B4ACF5AD1622
:10B82300949494B49CD59CF59CD58CB48C938CB394
:10B833007C32849374327C7384F57C947CB48D164F
:10B843008D178CD78CD78CD794D79CD89CF8A519F7
:10B85300A4F9AD19AD19AD192000000000000000D6
:10B8630000000000000000000022000000000000B3
:10B87300142828500000000000002C0000000000E5
:10B8830000181808300000000000002D0000000020
:10B8930000000000FE000000000000002E00000079
:10B8A3000000000018180000000000000030000035
:10B8B3000018244242424242422418000000310050
:10B8C30000001070101010101010107C00000032D7
:10B8D3000000003C42420204081020427E000000A7
:10B8E300330000003C42420418040242423C000080
:10B8F30000340000000808182848487E08081E0085
:10B903000000350000007E40405C62020242423C7F
:10B91300000000360000001C2440405C62424242AA
:10B923003C000000370000007E444408081010105B
:10B933001010000000380000003C4242423C244208
:10B9430042423C0000003900000038444242463A7B
:10B95300020224380000003A00000000001818001A
:10B9630000001818000000003B0000000008000061
:10B97300000000080810000000410000001010281B
:10B983002828287C4444EE00000042000000FC42CA
:10B9930042447844424242FC000000430000003E1F
:10B9A300428280808080824438000000440000008E
:10B9B300F84442424242424244F80000004500003B
:10B9C30000FC4248487848484042FC0000004600DA
:10B9D3000000FC4248487848484040E000000047E7
:10B9E3000000003C44848080808E84443800000042
:10B9F30048000000EE4444447C44444444EE0000C8
:10BA030000490000007C10101010101010107C0072
:10BA130000004A00003E08080808080808080888CB
:10BA2300F000004B000000EE44485070504848447A
:10BA3300EE0000004C000000E04040404040404029
:10BA430042FE0000004D000000EE6C6C6C54545438
:10BA53005454D60000004E000000EE646454545465
:10BA63004C4C4CE40000004F0000003844828282BA
:10BA7300828282443800000050000000FC424242AF
:10BA83007C40404040E00000005100000038448208
:10BA930082828282B24C3806000052000000F844D1
:10BAA30044447850484844E6000000530000003EF8
:10BAB300424240300C0242427C000000540000002D
:10BAC300FE921010101010101038000000550000E6
:10BAD30000EE4444444444444444380000005600C7
:10BAE3000000EE4444442828282810100000005782
:10BAF300000000D6545454546C2828282800000011
:10BB030058000000EE4428281010282844EE0000B6
:10BB13000059000000EE444428281010101038008B
:10BB230000005A0000003E44040808101020227E42
:10BB33000000005B00003C2020202020202020204B
:10BB430020203C0000004040202010101008080472
:10BB5300040402005D00003C04040404040404041F
:10BB63000404043C005E00000000000000182400F0
:10BB73000000000000005F0000000000000000FE65
:10BB83000000000000000060000000000000003022
:10BB930008000000000000006100000000003844BD
:10BBA3001C2444443E0000000062000000C04040EA
:10BBB3005C62424242427C000000630000000000DD
:10BBC3001C22404040221C00000000640000000CC6
:10BBD30004047C848484848C760000006500000067
:10BBE30000003C427E4040423C00000000660000F2
:10BBF300000E12107C10101010107C000000670063
:10BC03000000003E444438403C42423C000000688F
:10BC1300000000C040405C6242424242E700000034
:10BC2300690000003030007010101010107C00000C
:10BC3300006A00000C0C001C04040404040444788F
:10BC430000006B000000C040404E4850684844EE7E
:10BC53000000006C00000070101010101010101085
:10BC63007C0000006D0000000000F854545454544C
:10BC7300D6000000006E0000000000DC6242424279
:10BC830042E7000000006F00000000001824424259
:10BC9300422418000000007000000000DC624242F1
:10BCA30042427C40E000000071000000007C84847C
:10BCB30084848C74040E000000720000000000EE07
:10BCC3003220202020F80000000073000000000054
:10BCD3003C44403804447800000000740000000035
:10BCE30010107C10101010100C00000075000000E4
:10BCF3000000C642424242463B000000007600007C
:10BD0300000000E742242428101000000000770000
:10BD130000000000D654545428282800000000785E
:10BD230000000000006E241818182476000000009C
:10BD33007900000000E742242428181010E00000D6
:10BD4300007A00000000007E44081010227E0000EC
:10BD530000007B000018101010101020101010109D
:10BD63001018007C0010101010101010101010107C
:10BD7300101010107D00003010101010100810105B
:10BD830010101030007E0000000000000062928C52
:10BD930000000000000000C9EE400027FE2404015B
:10BDA30020811856085040104027FC2040C0E04135
:10BDB30058464E584440404040DBDA00001204121B
:10BDC300441244FE44124412441244124412443AAC
:10BDD30044C4440444080410040000CEB008400CDA
:10BDE30040084017FC104033FC3040504097FC1093
:10BDF30044104410441044105410481040C7B60176
:10BE03000021083FF80000244024407E7C24842540
:10BE1300283C20242024503C48248E25040200BFC3
:10BE2300C60608788808480848FE0818881C482A67
:10BE330048280E48788B8808080808080808080866
:10BE430008BCBC102010201020FDFE102014201967
:10BE5300FC3108D0881090106010601090110E56BD
:10BE6300042000B5E70100010001003FF82108218B
:10BE7300083FF82108210821083FF82108010201A1
:10BE83000200FE0000D7D300003FF0002000400076
:10BE930080010001000104FFFE0100010001000117
:10BEA30000010005000200D3D0010001007FFE0263
:10BEB3000004000FF0181028104FF0881008100F1E
:10BEC300F00810089008700820CFDE0000FBF892FD
:10BED3000893F8A208A20893F88A808A48AA509285
:10BEE3002082208210828E83048200B9AB0000047A
:10BEF3004006400440082008101018220E43040294
:10BF0300000420081011F83F1810100000CBBE00E9
:10BF1300003FFC000400047FE4000400043FC4204D
:10BF23004420443FC420442004001400080000C9F6
:10BF3300E4080810083F0821083FFE21083F0821B4
:10BF43004821287F280528090811082108452802C7
:10BF530010C6B5080008FE4E20484048FCFE840089
:10BF6300A408A44AA44AA484A4085010482086C361
:10BF7300020000BFA80100010001FC010001000153
:10BF8300007FFE01000100014001300118010C0196
:10BF93000801000100BDC92108320827C8445057D1
:10BFA300DEF47417D4211447D4F21403881A88E4F6
:10BFB3009404940AA61144B7D102403FF802483FC3
:10BFC300F822403FFE0442084A1FF4681009100992
:10BFD30010091002C00C383010CFB5007C3F80022E
:10BFE30020042008401F8003200C103FF8108C040D
:10BFF300A008901088208442840100CDB310401023
:10C003002023FE20404440F888090413FE20947C3A
:10C0130090009000901D12E112020E0400D3E00183
:10C023000001000280046008103FFEC10401003FCC
:10C03300FC0100114019301118211045000200B60F
:10C04300EE100008FE7F9051201EFE228254820CC7
:10C053009212923E92E29222AA22243E422182002E
:10C0630000BAC51FF01010101010101FF00000FFD1
:10C07300FE080008001FF008100010001001100057
:10C08300A00040D4AA00001FF80000000000007FB9
:10C09300FE0440044004400440084008401042208D
:10C0A30042403E0000B3F51000080008047EFE0481
:10C0B30024082412243424582494241244104410B1
:10C0C30084111412080000CABC102018301020106C
:10C0D30048FC8425FE2484440044FC2884188414EA
:10C0E30084228442FC80840000BBAF08800C80085B
:10C0F30088108C109830B050E090C01180128014DA
:10C1030080108410841084107C0000CAA7010009E9
:10C1130000090011001FF82100410001007FFE010A
:10C12300000280024004200830101C2008B0DC000C
:10C13300403E60224022802AFE2B882A882A882AB1
:10C143005008501420122023502288410E0204D696
:10C15300D801F03F000100FFFE01001FF011101F86
:10C16300F011101FF001003FF801000100FFFE0075
:10C1730000C6F4010000C000801FFC100410041F5F
:10C18300FC1000100017FC14042404240447FC844E
:10C19300040000D6D00100010021083FFC21082142
:10C1A300082108210821083FF821080100010001A6
:10C1B3000001000100B6C10040404033FC204007AD
:10C1C300FE0104E4A822A0222027FE2020205028DC
:10C1D30088310422060404C7EB004047FC304023A7
:10C1E300F8004007FEF00013F8120813F8120813C2
:10C1F300F816081A0812280210CBA23F82208220C8
:10C203009220923F92221222125FD25252525252E3
:0BC21300525252524293C2028A0204AF
:10E0AA00420059020349004F0931000004110011CE
:10E0BA000045004805300000041A401A220004FFF7
:10E0CA00FFFFFFFFFF060000000000000000000045
:05E0DA00010203040532
:0BE2B000EF1FAC0670011E4C70F62240
:0BE1FA007C007E0012E27B7F327E0082
:10E20500AB07AA06EB1BAE0270011A4E60097F959B
:08E215007E0012E2B080ED2250
:10E25C00AD07AC06C2A5C2A4ECF580C2A3D2A3ED57
:09E26C00F580C2A3D2A3D2A522C1
:05E23E00E0FEA3E0FF7B
:10E24300AD07AC06C2A5D2A4ECF580C2A3D2A3ED60
:09E25300F580C2A3D2A3D2A522DA
:10E21D0090000EE0FBA3E475F00112C8ABA9F0FA73
:04E22D0012C81BFFF9
:0DE23100C2A5D2A48F80C2A3D2A3D2A52281
:07E2BB00901C00E0FF7E0053
:01E2C2002239
:06E275007D077C007E0025
:0EE27B00AB05AA0412E25CAE02AF0302E2435E
:10D43500C2A1C2A67F0A7E0012E205D2A67D087CA3
:10D44500307FE37E0012E27B7D127C007FE77E0069
:10D4550012E27B7D317C127FEF7E0012E27B7D0044
:10D465007C017F017E0012E27B7D007C077F027ECE
:10D475000012E27B7D307C107F037E0012E27BE4AC
:10D48500FDFC7F04FE12E27B7D077C027F087E00A7
:10D4950012E27B7D007C077F097E0012E27BE4FDC2
:10D4A500FC7F0AFE12E27BE4FDFC7F0CFE12E27BB0
:10D4B500E4FDFC7F0DFE12E27BE4FDFC7F0FFE1216
:10D4C500E27B7DF07C007F107E0012E27B7F1112F3
:10D4D500E2757D967C007F127E0012E27BE4FDFC06
:10D4E5007F13FE12E27B7FC87E0012E2057D907CF1
:10D4F500147F107E0012E27B7D277C027F1112E1F2
:10D50500FC7D1D7F1212E1FA7D007C1A7F137E00DF
:10D5150012E27B7D337C007F297E0012E27B7D0E4B
:10D525007F2B12E1FAE4FDFC7F20FE12E27BE4FD95
:10D53500FC7F21FE12E27B7F3012E2757D067C02C4
:10D545007F317E0012E27B7D067C057F327E0012F4
:10D55500E27B7D047C077F357E0012E27B7D037CC8
:10D56500127F367E0012E27B7D077C007F377E00CE
:10D5750012E27BE4FDFC7F38FE12E27B7D067C0730
:10D585007F397E0012E27B7D017C077F3C7E0012A5
:10D59500E27B7D0F7C007F3D7E0012E27BE4FDFC9B
:10D5A5007F50FE12E27B7DEF7C007F517E0012E210
:10D5B5007BE4FDFC7F52FE12E27B7D3F7C017F53C5
:10D5C5007E0012E27B7D007CA77F607E0012E27BFD
:10D5D5007D017C007F617E0012E27BE4FDFC7F6AB9
:10D5E500FE12E27B7D107C007F907E0012E27B7D47
:10D5F500007C067F927E0012E27B7D037C007F9398
:10D605007E0012E27B7D107C017F957E0012E27B1D
:10D61500E4FDFC7F97FE12E27BE4FDFC7F98FE12A1
:10D62500E27B7D337C017F077E0012E27B7F647E97
:10D635000012E205D2A190004D74FFF0A374E0F052
:0AD6450090005B74F8F0A3E4F022FB
:05E13A002DFDE03CFC9E
:10E13F008D828C83AD07AC067F207E0012E27BAE12
:10E14F0083AF82AD07AC067F217E0012E27B7F2278
:05E15F007E0002E25CFD
:10DFA600900028EEF0A3EFF0A3ECF0A3EDF0A3EAC7
:10DFB600F0A3EBF0900028E0FCA3E0FD7F507E008C
:10DFC60012E27B90002CE0FCA3E0FD7F517E001264
:10DFD600E27B90002AE0FCA3E0FD7F527E0012E285
:10DFE6007B90002EE0FCA3E0FD7F537E0012E27BD7
:10DFF600900028E0FEA3E0FFA3E0FCA3E0FD02E121
:01E006003FDA
:10DD860090000CE4F0A374E7F074FFA3F0A3F07D19
:0BDD9600C87BE67A007C007F787E00EE
:10DDA100900006EEF0A3EFF0A3ECF0A3EDF0A3EAF0
:04DDB100F0A3EBF000
:10DDB500C007A3E0FFA3E090002ECFF0A3EFF0D0C3
:10DDC5000712DFA6900008E0FFA3E0900010CFF057
:10DDD500A3EFF090000CE0FEA3E0FFD3900011E06C
:10DDE5009F900010E09E5034900006E0FEA3E0FBFB
:10DDF500AA06C390000BE09B90000AE09A400D90A4
:10DE0500000E12E23E0BBB00010A80E6900011E015
:0CDE150004F070BF900010E004F080B733
:01DE210022DE
:10E18B0090000C7401F0A37440F090005BE0FFA3CF
:10E19B00E090000ECFF0A3EFF07BF07A00E4FDFCF3
:05E1AB00FFFE02DDA1F2
:08E00700900003EEF0A3EFF01E
:10E00F0090002E7401F0A3743FF07BEF7A00E4FDD3
:10E01F00FCFFFE12DFA6E4FDFCFFFE12E13FE490E1
:10E02F000005F0A3F0E4FBFA90000312E23E0BBBF5
:10E03F0000010ABA01F2BB40EF900006E004F07055
:10E04F0006900005E004F0C3900006E094F0900005
:06E05F0005E0940040CF33
:01E065002298
:0ED9F500900012EEF0A3EFF0A3ECF0A3EDF023
:10DA0300E490001EF0A3F0A3F0A3F0A3F0A3F0A30F
:10DA1300F0A3744FF0E490001EF0A3F090001EE01A
:10DA2300FEA3E0FFC3944FEE9400502C12C81BFDDD
:10DA330090B85B75F011EF12C90BEE75F011A425C8
:10DA430083F583E4936D601090001FE004F070CCC5
:10DA530090001EE004F080C4900024E0FEA3E0FFE9
:10DA6300C390001FE09F90001EE09E400302DB79FD
:10DA7300900012E0FAA3E0FBFFAE02C006C007A3CA
:10DA8300E0FCA3E0FDEB2407FBE43AFA900014E08A
:10DA9300FEA3E0240FFFE43E90002EF0A3EFF0D0AE
:10DAA30007D00612DFA6E4900020F0A3F090002038
:10DAB300E0FEA3E0FFC39410EE9400400302DB7981
:10DAC30090001EE0FCA3E090B85C75F01112C90B46
:10DAD300EC75F011A42583F583E5822FF582E583A8
:10DAE3003EF583E493F9E4900022F0A3F090002242
:10DAF300E0FEA3E0FFC39408EE9400506874807EB8
:10DB030000A807088006CEA2E713CE13D8F8FFE9D2
:10DB1300FDEF5D6005900019800990001DE070081D
:10DB230090001B12E23E802C900022E0FEA3E0FF57
:10DB3300900013E02FFF900012E03ECF2401CF347A
:10DB430000FE900020E0FCA3E0FD900015E09000B3
:10DB53001412E13A900023E004F07091900022E067
:10DB630004F002DAF0900021E004F0700690002047
:06DB7300E004F002DAB04C
:01DB79002289
:0ED64F00900012EEF0A3EFF0A3ECF0A3EDF0CC
:10D65D00E490001EF0A3F0A3F0A3F0A3F0A3F090CC
:10D66D000026F0A37422F0E490001EF0A3F09000C9
:10D67D001EE0FEA3E0FFC39422EE9400505112C8A9
:10D68D001BFD90BD9A75F022EF12C90BEE75F022BD
:10D69D00A42583F583E493B5052590000112C834C4
:10D6AD00FF90001EE0FCA3E090BD9B75F02212C917
:10D6BD000BEC75F022A42583F583E4936F60109035
:10D6CD00001FE004F070A790001EE004F0809F9012
:10D6DD000026E0FEA3E0FFC390001FE09F90001E18
:10D6ED00E09E400302D83F900012E0FAA3E0FBFF5A
:10D6FD00AE02C006C007A3E0FCA3E0FDEB240FFBC8
:10D70D00E43AFA900014E0FEA3E0240FFFE43E900B
:10D71D00002EF0A3EFF0D007D00612DFA6E49000A4
:10D72D0020F0A3F0900020E0FCA3E0FD25E0FFEC4D
:10D73D0033FE90001EE0FAA3E090BD9C75F022121E
:10D74D00C90BEA75F022A42583F583E5822FF582B6
:10D75D00E5833EF583E493FAED25E0FFEC33FE908F
:10D76D00001EE0FCA3E090BD9D75F02212C90BECEC
:10D77D0075F022A42583F583E5822FF582E5833E9E
:10D78D00F583E493FFEAFE900024EEF0A3EFF0E4BE
:10D79D00900022F0A3F0900022E0FEA3E0FFC394DE
:10D7AD0010EE9400506CE47E80A807088005CEC36F
:10D7BD0013CE13D8F9FF900024E05EFEA3E05F4E78
:10D7CD006005900019800990001DE0700890001B05
:10D7DD0012E23E802C900022E0FEA3E0FF900013A9
:10D7ED00E02FFF900012E03ECF2401CF3400FE90D9
:10D7FD000020E0FCA3E0FD900015E090001412E184
:10D80D003A900023E004F07006900022E004F0024C
:10D81D00D7A3900021E004F07006900020E004F002
:10D82D00C3900021E09410900020E094005003027A
:02D83D00D731E1
:01D83F0022C6
:10DC94007BFF90000D7407F074E0A3F0A37407F009
:0DDCA400A374E0F0E4A3F07D96FC7F2DFE5C
:10DCB100900006EEF0A3EFF0A3ECF0A3EDF0A3EBE0
:10DCC100F0A3EAF0A3E9F090000AE0FBA3E0FAA3D5
:10DCD100E0F912C81BFF700302DD85EFD394809039
:10DCE1000008E0FCA3E0FD404890000DE0FFA3E048
:10DCF100900019CFF0A3EFF090000FE0FFA3E090A8
:10DD0100001BCFF0A3EFF0900011E090001DF09008
:10DD11000006E0FEA3E0FF12D64F900007E02410BA
:10DD2100F0900006E03400F090000BE475F0028002
:10DD31004DA3E0FBA3E0FAA3E0F9A3E0FFA3E09089
:10DD41000019CFF0A3EFF090000FE0FFA3E09000E7
:10DD51001BCFF0A3EFF0900011E090001DF09000B8
:10DD610006E0FEA3E0FF12D9F5900007E02408F0D9
:10DD7100900006E03400F090000BE475F00112C849
:05DD81009502DCC82240
:10CEAE00900033EEF0A3EFF0A3ECF0A3EDF0A3EAC5
:04CEBE00F0A3EBF002
:10CEC200FFAE02E4FCFD7B807A967998F812E06668
:10CED200EF243090003FF0900037E0FEA3E0FFE443
:10CEE200FCFD7B807A967998F812E066AC00AD0181
:10CEF200AE02AF037B407A42790F780012E066EF10
:10CF02002430900040F0900037E0FEA3E0FFE4FC04
:10CF1200FD7B807A967998F812E066AC00AD01AE9E
:10CF220002AF037B407A42790F780012E066AC00D0
:10CF3200AD01AE02AF037BA07A867901780012E0E0
:10CF420066EF2430900041F0900037E0FEA3E0FF4E
:10CF5200E4FCFD7B807A967998F812E066AC00AD2D
:10CF620001AE02AF037B407A42790F780012E0668D
:10CF7200AC00AD01AE02AF037BA07A8679017800E6
:10CF820012E066AC00AD01AE02AF03E47B107A277B
:10CF9200F9F812E066EF2430900042F0900037E09A
:10CFA200FEA3E0FFE4FCFD7B807A967998F812E01C
:10CFB20066AC00AD01AE02AF037B407A42790F78D6
:10CFC2000012E066AC00AD01AE02AF037BA07A8630
:10CFD2007901780012E066AC00AD01AE02AF03E465
:10CFE2007B107A27F9F812E066AC00AD01AE02AF11
:10CFF20003E47BE87A03F9F812E066EF243090004C
:10D0020043F0900037E0FEA3E0FFE4FCFD7B807A72
:10D01200967998F812E066AC00AD01AE02AF037BE0
:10D02200407A42790F780012E066AC00AD01AE02A0
:10D03200AF037BA07A867901780012E066AC00AD7E
:10D0420001AE02AF03E47B107A27F9F812E066AC76
:10D0520000AD01AE02AF03E47BE87A03F9F812E017
:10D0620066AC00AD01AE02AF03E47B64FAF9F812DC
:10D07200E066EF2430900044F0900037E0FEA3E039
:10D08200FFE4FCFD7B807A967998F812E066AC00AA
:10D09200AD01AE02AF037B407A42790F780012E015
:10D0A20066AC00AD01AE02AF037BA07A867901784F
:10D0B2000012E066AC00AD01AE02AF03E47B107A71
:10D0C20027F9F812E066AC00AD01AE02AF03E47BD3
:10D0D200E87A03F9F812E066AC00AD01AE02AF03E4
:10D0E200E47B64FAF9F812E066AC00AD01AE02AF7F
:10D0F20003E47B0AFAF9F812E066EF243090004567
:10D10200F0900037E0FEA3E0FFE4FCFD7B807A961E
:10D112007998F812E066AC00AD01AE02AF037B4035
:10D122007A42790F780012E066AC00AD01AE02AF30
:10D13200037BA07A867901780012E066AC00AD012B
:10D14200AE02AF03E47B107A27F9F812E066AC0076
:10D15200AD01AE02AF03E47BE87A03F9F812E066B0
:10D16200AC00AD01AE02AF03E47B64FAF9F812E061
:10D1720066AC00AD01AE02AF03E47B0AFAF9F81225
:10D18200E066EB2430900046F0E4A3F090003EF01D
:10D1920090003EE0FFC394095075743F2FF582E47E
:10D1A2003400F583E024D0700890003EE0640870FB
:10D1B2005690003EE0FB75F004A4FF900034E02F8F
:10D1C200FF900033E035F0FEC007900035E0FCA38D
:10D1D200E0FD743F2BF9E43400FA7B01900039E062
:10D1E200FFA3E090000DCFF0A3EFF090003BE0FF33
:10D1F200A3E090000FCFF0A3EFF090003DE090008D
:0FD2020011F0D00702DCB190003EE004F0808113
:01D2110022FA
:06DEAE007A007C007E00FA
:10DEB400900006EEF0A3EFF0A3ECF0A3EDF0A3EADC
:04DEC400F0A3EBF0EC
:10DEC800E4900011F0A3F090000CE0FEA3E0FFC383
:10DED800900012E09F900011E09E504D900006E0E7
:10DEE800FEA3E0FF900011E0FCA3E0FD900009E034
:10DEF8002DFD900008E03CFC12E13FE4FDFCD390CE
:10DF0800000BE09D90000AE09C400D12E21D12E219
:10DF18001D0DBD00010C80E6900012E004F070A712
:09DF2800900011E004F002DECFCC
:01DF310022CD
:10D8400090000374FFF0A37400F0A374C3F0900081
:10D850000CE4F0A37446F0900003E0F9A3E0FAA30F
:10D86000E090000EC9F0A3EAF0A3E9F07BF07A00A3
:10D87000E4FDFCFFFE12DEB490000CE4F0A3745D46
:10D88000F0A374F8F0A3E4F07BEFFA7D46FCFFFE12
:10D8900012DDA17BFF7A00790390000D74FFF0A3E5
:10D8A00074E0F0A374F8F0A3E4F0A3F07D4AFC7FE9
:10D8B00026FE12DCB190000C7401F0A3743FF0A3BB
:10D8C0007407F0A374E0F07BEF7A007D5E7C00E4E7
:10D8D000FFFE12DDA190000374FFF0A37497F0A384
:10D8E000748BF090000CE4F0A37414F0900003E04B
:10D8F000F9A3E0FAA3E090000EC9F0A3EAF0A3E9CF
:10D90000F07B787D6E7F7812DEAE7BFF7A0079182F
:10D91000E490000DF0A3F0A37407F0A374E0F0E42A
:10D92000A3F07D86FC7F8CFE12DCB190000374FFB7
:10D93000F0A37484F0A37403F090000CE4F0A374DB
:10D9400032F0900003E0F9A3E0FAA3E090000EC9E2
:10D95000F0A3EAF0A3E9F07B327DB47F0F12DEAED4
:10D9600090000374FFF0A374AAF0A3744BF090002E
:10D970000CE4F0A3741EF0900003E0F9A3E0FAA316
:10D98000E090000EC9F0A3EAF0A3E9F07B3C7A0036
:10D990007DEC7C007F0A7E0012DEB412DD869000F2
:10D9A0000C7401F0A3740BF074FFA3F0A3F07DECF2
:10D9B00012DD977BFF7A007921E490000DF0A3F04F
:10D9C000A37407F0A374E0F0E4A3F07DD0FC7F50D3
:10D9D000FE12DCB17BFF7A007926E490000DF0A303
:10D9E000F0A37407F0A374E0F0E4A3F07DF4FC7FEF
:05D9F00050FE02DCB155
:0CE29800EF4E6007EF1F70F81E80F522AB
:08E0E000789CA6077F647E0016
:10E0E80075CBFC75CA6975CDFC75CC69C2AD75C8B0
:10E0F80004EF1FAC0670011E4C600730CFFDC2CF85
:05E1080080EFC2CA22F5
:10E10D0075CBDC75CA0075CDDC75CC00C2AD75C89C
:10E11D0004EF1FAC0670011E4C600F20CF08300AB3
:0DE12D00FAC2CAC2CF22C2CF80E7C2CA2206
:10E1B000750808AD081508ED6016EE2EFEC295EF45
:10E1C000339297EF2FFFA296E4334EFED29580E371
:04E1D000D295AF062F
:01E1D4002228
:0EE28900C2937FAA12E1B07FFF12E1B0D293E0
:01E297002264
:0DDB7A007F647E0012E0E87B007A007922D3
:0BDB8700900003EBF0A3EAF0A3E9F02C
:10DB9200E4900007F0900006F0900006E0FCC394C9
:10DBA20064501912E289EFB4F00374FDF07F0A7E2B
:10DBB2000012E298900006E004F080DDEC64FE6062
:10DBC2000302DC91C2937FBB12E1B0900006EFF03A
:10DBD200900003E0FBA3E0FAA3E0F9740112C8612C
:10DBE200E4900006F0900003E0FBA3E0FAA3E0F962
:10DBF20012C81BFF900006E0C39F50457FFF12E151
:10DC0200B0900003E0FBA3E0FAA3E0F9A3E0FEF585
:10DC120082758300EF12C873900007E0FF8E827551
:10DC2200830012C834FEEF6E900007F012C81BD3B7
:10DC320094204005D2937F0122900006E004F080F8
:10DC4200A47F0A7E0012E0E87FFF12E1B090000399
:10DC5200E0FBA3E0FAA3E0F9A3E0F582758300EF0D
:10DC620012C8737F0A7E0012E0E8D293900003E0AC
:10DC7200FBA3E0FAA3E0F9A3E0F58275830012C8E2
:10DC820034FF900007E0B507037F00227F01227F67
:01DC92000190
:01DC9300226E
:10DF3200784A7C007D007B007A00799F7E007F0416
:10DF420012C7F57B007A007940900000EBF0A3EA5B
:04DF5200F0A3E9F05F
:0BDF5600900003EBF0A3EAF0A3E9F059
:10DF6100E4A3F0C2937FCC12E1B0E4FC900003E0A3
:10DF7100FBA3E0FAA3E0F912C81BFEECC39E501A02
:10DF8100900006E0FE8C8275830012C834FFEE6FAC
:10DF9100900006F012E1B00C80D2900006E0FF1272
:04DFA100E1B0D29386
:01DFA5002259
:0CE2A400C2927F327E0012E10DD2922265
:10D21200E4789DF608F60812C8F24352800012E143
:10D22200D512E2A47FF47E0112E0E812D435E4FFC5
:10D23200FE12E00712D8402094FD12DF3212DB7A90
:10D24200789CA607900000E0FBA3E0FAA3E0F99027
:10D25200000112C834FF7823E6B50705789CE66022
:10D262000B12DF4512DB7A12E0E080D8789EE6648A
:10D27200011846700302D4342094FD7F507E0012C0
:10D28200E0E82094E77BFF7A00797912DF4B12DB2A
:10D292007A789CA607900000E0FBA3E0FAA3E0F9ED
:10D2A20090000112C834FF7823E6B50705789CE6A2
:10D2B200602E7BFF7A0079C112DF56789CA6077B2D
:10D2C200FF7A00792B90000DE4F0741F12DC9E7F30
:10D2D200F47E0112E0E87A00793C12DC9402D284F6
:10D2E200789F7C007D007B007A0079247E007F0499
:10D2F20012C7F5789F12C8C1E4FBFA79C078BF1251
:10D30200C225789F12C8DAE4FFFEFDFC789F12C89E
:10D31200CD12C31650367BFF7A0079C112DF5678E0
:10D322009CA6077BFF7A00794D90000DE4F0A37470
:10D332001F12DC9F7FF47E0112E0E87A0079581216
:10D34200DC94789D760008760102D26E12DF3212EA
:10D35200DB7A789CA607900000E0FBA3E0FAA3E04A
:10D36200F990000112C834FF7823E6B50705789CCE
:10D37200E6600B12DF4512DB7A12E0E080D8900003
:10D382000674FFF0A37400F0A37464F0789F12C8CF
:10D39200C190000912C8E67B007A00797C12CA901B
:10D3A2007BFF7A0079C112DF5612E0E07BFF7A0040
:10D3B200796AE490000DF0A3F074FFA3F0A3F0E407
:10D3C200A3F07DD0FC7F7DFE12DCB17B007A007978
:10D3D2007CE490000DF0A3F074FFA3F0A3F0E4A3AB
:10D3E200F07DF4FC7F7DFE12DCB17BFF7A00797365
:10D3F200E490000DF0A3F074FFA3F0A3F0E4A3F017
:10D402007DF4FC7FB4FE12DCB17FC47E0912E0E839
:10D4120012DD8690000C7401F0A3740BF074FFA36C
:10D42200F0A3F07BE67A007DEC12DD9B12DD860232
:02D43200D284A2
:01D4340022D5
:10E1D500C2AD75C804758780759870758921758D70
:10E1E500FD858D8BD28EC2ABD2AFC2A8D288C2CAF2
:05E1F500D2ACC20A22B9
:10C21E0002C3B8E86480F8E933E83360110460F0D3
:10C22E00ED33EC337009E8FCE9FDEAFEEBFF220486
:10C23E0060DED3EB9FEA9EE99DE8C2E78CF0C2F781
:10C24E0095F0400CE8CCF8E9CDF9EACEFAEBCFFB4D
:10C25E0012C38385D0F05804700320D5B3E8047060
:10C26E00075002B2D502C3C292D5EC0460F7E4CCFB
:10C27E00C0E0C398F8603B94186008400DD0E0FB16
:10C28E0002C39AE4FBFAC9FC8028E830E406E4C94C
:10C29E00FBE4CAFCE830E305E4C9CACBFCE854076A
:10C2AE006010F8C3E913F9EA13FAEB13FBEC13FC75
:10C2BE00D8F130F52FC3E49CFCEF9BFFEE9AFEED18
:10C2CE0099FDD0E0FBEF4E4D4C701222DB0302C302
:10C2DE00BFEC2CFCEF33FFEE33FEED33FDED30E71C
:10C2EE00EB02C39AEF2BFFEE3AFEED39FDD0E0FBE9
:10C2FE0050130BBB000302C3C2ED13FDEE13FEEF92
:08C30E0013FFEC13FC02C39ABB
:10C3160074F8CC6480CCC86480C8F582046043C3DA
:10C32600EB9FF5F0EA9E42F0E99D42F0E89C45F06D
:10C3360060305018E5825FFFE582F42B5582FB5092
:10C34600210ABA001D09B90019088016E5825BFBAF
:10C35600E582F42F5582FF50090EBE00050DBD0083
:10C36600010CC3EB9FF5F0EA9E42F0E99D42F0E82E
:0DC376009C45F06007CC4820E701B3EC22A5
:10CA2B00E5082406F582E43400F583E0050822903E
:10CA3B000003300703900006E475F00112C91702DA
:10CA4B00C81B2000E97F2ED2008018EF540F2490D2
:10CA5B00D43440D4FF30040BEF24BFB41A0050037E
:10CA6B002461FFE50960021509050CE50C70020550
:10CA7B000B30070E900003E475F00112C917EF029B
:10CA8B00C86102E1647403D2078003E4C207F508AE
:10CA9B0090000312C92EE4F509F50BF50CE50960BE
:10CAAB00077F2012CA6E80F5750AFFC201C200C251
:10CABB0002C203C205C206C20812CA3AFF700D3089
:10CACB0007057F0012CA7FAF0CAE0B22B4255FC2E5
:10CADB00D5C20412CA3AFF24D0B40A00501A75F01A
:10CAEB000A780930D50508B6FF0106C6A426F6203C
:10CAFB00D5047002D20380D924CFB41A00EF5004AE
:10CB0B00C2E5D20402CD71D20180C6D20080C0D260
:10CB1B000280BCD2D580BAD20580B47F2012CA6EF7
:10CB2B002002077401B5090040F112CA2BFF12CA8B
:10CB3B006E02CAA8D208D206809512CA2BFB12CA63
:10CB4B002BFA12CA2BF94A4B7006796F7ACE7BFF00
:10CB5B0020022EE509602A7E008E8275830012C8A2
:10CB6B003460060EEE650A70F0C2D5EBC0E0EAC089
:10CB7B00E0E9C0E0EE12CDD2D0E0F9D0E0FAD0E09F
:10CB8B00FB12C81BFF60AAEBC0E0EAC0E0E9C0E003
:10CB9B0012CA6ED0E02401F9D0E03400FAD0E0FBE9
:10CBAB00E50A0460DCD50AD98087D20280A212CDB7
:10CBBB00B460F7E50A70010412C3CDA90A600DE554
:10CBCB000A600914F50A12CE5CEF60F3EA30E70253
:10CBDB00F404C3995079EAF4250A0430E701E4041C
:10CBEB00F50A800D12CDB460C1EA050A250A12C3FD
:10CBFB00CDEA900032F030E701E4250A04D50A04AF
:10CC0B002005011412CDD2E4C0E012CE5C900032AC
:10CC1B00E0601320E70714F012CA56802204F0D00C
:10CC2B00E014C0E07F0012CA56E50A600712CA4D35
:10CC3B00150A800B30050312CA4DD0E002CAA8D0EA
:10CC4B00E00480C412CDB4609EE50A0412C3CD90FB
:10CC5B000032EAF0E50A200502600104240412CD3B
:01CC6B00D2F6
:10CC6C0074FF04C0E012CE5C12CA56E50A2005021D
:10CC7C00600312CA4DD0E0B50AE87F4512CA609035
:10CC8C000032E07F2B30E7047F2DF404C0E012CAA1
:10CC9C006ED0E075F00A84C0F012CA57D0E012CA08
:10CCAC005702CAA8791080027908C206C208800807
:10CCBC00D2D5790A8004790AC2D5E50A047002F546
:10CCCC000AE4FAFDFEFF12CA2BFC7B0820011312AA
:10CCDC00CA2BFD7B1030000A12CA2BFE12CA2BFF86
:10CCEC007B20EC3382D592D55013C3E43000069FE1
:10CCFC00FFE49EFEE42001039DFDE49CFCE4CBF8E4
:10CD0C00C201EC700CCFCECDCCE824F8F870F380D7
:10CD1C0017C3EF33FFEE33FEED33FDEC33FCEB3397
:10CD2C00FB994002FB0FD8E9EB300105F8D0E0C4C9
:10CD3C0048B201C0E00AEC4D4E4F78207B0070C227
:10CD4C00EAB50A0040BCC0E012CDD4D0F0D0E0204F
:10CD5C000104C4C0E0C4B201C0F012CA57D0F0D56F
:10CD6C00F0EB02CAA812C937CB4553CCB058CB163E
:10CD7C004CCB1242CCB44FCCBC44CCBC49CB2B4397
:10CD8C00CCC255CBEF46CC4F45CBB947CE8F50CB11
:10CD9C001A2DCB1E2ECB412BCB2223CB3F20CE7872
:10CDAC002ACADA480000CB39E50AB4FF03750A0633
:10CDBC0012CA2BFC12CA2BFD12CA2BFE12CA2BFF55
:10CDCC0090002B02C40A790AA2D52003143005095D
:10CDDC00B910020404B9080104A2D52006025001BE
:10CDEC00042002689202B509005034C0E07F203064
:10CDFC0003197F30A20272067205500F12CE2BC29D
:10CE0C0002C206C205C2087F30800F300503E9C09C
:10CE1C00E012CA6E300503D0E0F9D0E0B509CC3091
:10CE2C0005177F30B9100C12CA6E7F583004077F7B
:10CE3C00788003B9080312CA6E3002057F2D02CA2E
:10CE4C006E7F202008F87F2B2006F322920280CFE1
:10CE5C007F00B40700500B242BF582E43400F583DB
:10CE6C00E0FF22286E756C6C2900D20112CA2B309F
:10CE7C0001F8C201780930D50108F602CADA2D5042
:10CE8C0043495812CA2B2403B405004001E490CE48
:10CE9C008A9312CA5F743A12CA5FD20375090402EC
:02CEAC00CCB008
:10C38300E9D2E7C933E833F892D5EDD2E7CD33EC00
:07C3930033FC5002B2D52279
:10C39A00EC30E7100FBF000C0EBE00080DBD000404
:10C3AA000BEB6014A2D5EB13FCED92E7FD2274FFB0
:10C3BA00FCFDFEFF22E480F8A2D574FF13FC7D8009
:03C3CA00E480EF1D
:10C3CD00F920E73624F950037907E4F42402FBE55C
:10C3DD0082158270021583DBF6E024FB501BE960A9
:10C3ED0014E4F0E582158270021583E004F0B40ABE
:0DC3FD0008E4F0D9EE7401F00A22C2D52246
:10C40A00ED33EC3392D5FA602AB4FF33EDC2E77B01
:10C41A00FF60067AC4792FE4227AC4793820D504D9
:10C42A007AC47933224E614E002B494E46002D497B
:10C43A004E4600E47A08F0A3DAFC7B00740722C0B7
:10C44A0083C082ECC0E0EDC0E0EEC0E0EFC0E0EAFD
:10C45A0075F010A4CAABF075F04DA42BFBE435F0CF
:10C46A00FCEA2410FAEB34C5FBEC34D9FCEDC2E744
:10C47A00FF75F056A4F42411C5F0F434C58FF0A466
:10C48A002AE5F03BE43CF020E71412C6E5D0E0FFD1
:10C49A00D0E0FED0E0FDD0E0FC12C6188014F4040F
:10C4AA0012C6E5D0E0FFD0E0FED0E0FDD0E0FC12FD
:10C4BA00C50FD082D083E0FAEDD2E7CD33EC332436
:10C4CA0082FBE4C3CF33CFCE33CECD33CD33DBF3D0
:10C4DA007B0775F00A846004F0A31B0AE5F0F0A359
:10C4EA008FF0740AA4FFACF08EF0740AA42CFEAC90
:10C4FA00F050010C8DF0740AA42CFDE435F0F0A381
:05C50A00DBDE740722D6
:10C50F00EC4D6011E8497017ED33EC3304600DE426
:10C51F00FCFFFEFD22E933E8330470F802C3B812C2
:10C52F00C38358046009E4CC2481500628500902C3
:10C53F00C3C228400302C3BFC0E0EB4A7044B980B6
:10C54F0006D0E0FB02C3AEEF4E701CBD8008EBFFC0
:10C55F00EAFEE9FD80EBE98DF0A4FEE5F002C5F8F7
:10C56F00E9CDF9EAFEEBFFEF89F0A4FCE5F0CE8907
:10C57F00F0A42EFFE435F0CD89F0A42DFEE435F0C4
:10C58F008067EF4E7005BD80D780C3EF8BF0A4ACF2
:10C59F00F0EE8BF0A42CFCE435F0F8EF8AF0A42C2D
:10C5AF00E5F038FCE433CB8DF0A42CFCE5F03BF840
:10C5BF00EE8AF0A42CFCE5F038F8E433CF89F0A430
:10C5CF002CFCE5F038CF3400CE89F0A42FFFE5F036
:10C5DF003EFEE433C98DF0A42EFEE5F039CD8AF08E
:10C5EF00A42FFFE5F03EFEE43DFD33D0E0FB500706
:10C5FF000BBB000F02C3C2EC2CFCEF33FFEE33FE7C
:06C60F00ED33FD02C39AA9
:10C6150002C3C2EC5D046005E85904700302C3B8A7
:10C6250012C383580460F6EC4860F2EC7004FDFE1A
:10C63500FF22C860DB2481C85009C39860025006F8
:10C6450002C3BF9850CAF582E9294B4A7005AB82EF
:10C6550002C3AE75F0007C1A7880C3EF9BEE9AEDAD
:10C6650099400DC3EF9BFFEE9AFEED99FDE842F070
:10C67500DC23ACF0D0E0FFD0E0FED0E0FDAB8220C3
:10C68500E7101BEB60BAEC2CFCEF33FFEE33FEED4D
:10C6950033FD02C39AE803F830E705C0F075F000F2
:10C6A500EF2FFFEE33FEED33FD40B830E7C280AA31
:10C6B5003F8000004120000042C80000447A00008D
:10C6C500461C400047C35000497424004B1896800F
:10C6D5004CBEBC205A0E1BCA6753C21C749DC5AE06
:10C6E500FB60065407601C232312C713EB54386004
:10C6F5000912C6FF12C70E12C50FECF8EDF9EEFAD6
:10C70500EFCB22EB12C70E80F1543803241C90C6E0
:10C71500B5FE93FC0EEE93FD0EEE930ECE93FF2227
:0300000002DE22FB
:0CDE2200787FE4F6D8FD7581A202DE696D
:10C72500E709F608DFFA8046E709F208DFFA803EF6
:10C7350088828C83E709F0A3DFFA8032E309F608E3
:10C74500DFFA8078E309F208DFFA807088828C834B
:10C75500E309F0A3DFFA806489828A83E0A3F608FF
:10C76500DFFA805889828A83E0A3F208DFFA804CD9
:10C7750080D280FA80C680D4806980F280338010B0
:10C7850080A680EA809A80A880DA80E280CA803319
:10C7950089828A83ECFAE493A3C8C582C8CCC58391
:10C7A500CCF0A3C8C582C8CCC583CCDFE9DEE78061
:10C7B5000D89828A83E493A3F608DFF9ECFAA9F0E0
:10C7C500EDFB2289828A83ECFAE0A3C8C582C8CC36
:10C7D500C583CCF0A3C8C582C8CCC583CCDFEADE4F
:10C7E500E880DB89828A83E493A3F208DFF980CCB1
:10C7F50088F0EF60010E4E60C388F0ED2402B404AA
:10C805000050B9F582EB2402B4040050AF23234550
:06C81500822390C7757339
:10C81B00BB010689828A83E0225002E722BBFE021B
:09C82B00E32289828A83E493224E
:10C83400BB010CE58229F582E5833AF583E02250B9
:10C8440006E92582F8E622BBFE06E92582F8E22203
:0DC85400E58229F582E5833AF583E493221D
:10C86100BB010689828A83F0225002F722BBFE01B6
:02C87100F322B0
:10C87300F8BB010DE58229F582E5833AF583E8F0FB
:10C88300225006E92582C8F622BBFE05E92582C8A7
:02C89300F2228F
:10C89500C5F0F8A3E028F0C5F0F8E582158270022E
:06C8A5001583E038F022CB
:10C8AB00A3F8E0C5F025F0F0E58215827002158340
:06C8BB00E0C838F0E8229D
:10E06600C2D5E830E70FB2D5E4C39BFBE49AFAE4E5
:10E0760099F9E498F8EC30E717B2D512E09C12C98A
:10E0860099E4C39BFBE49AFAE499F9E498F88003CF
:10E0960012C99930D50DE4C39FFFE49EFEE49DFDB1
:04E0A600E49CFC22D8
:0CC8C100E6FC08E6FD08E6FE08E6FF22A3
:0DC8CD00E6FB08E6F908E6FA08E6CBF822DB
:0CC8DA00ECF608EDF608EEF608EFF6228A
:0CC8E600ECF0A3EDF0A3EEF0A3EFF022C5
:10C8F200D083D082E493F608740193F6087402930D
:09C90200F608740393F674047343
:0CC90B00A42582F582E5F03583F5832237
:10C91700F8E0FBA3A3E0F925F0F0E58215827002A9
:07C927001583E0FA38F0224D
:09C92E00EBF0A3EAF0A3E9F0220A
:10C93700D083D082F8E4937012740193700DA3A38F
:10C9470093F8740193F5828883E4737402936860A3
:06C95700EFA3A3A380DFA3
:10E16400EFB40A07740D12E16F740A309811A8997C
:10E17400B8130CC2983098FDA899C298B811F6301B
:07E1840099FDC299F59922F3
:10DE2E0002D212E493A3F8E493A34003F68001F226
:10DE3E0008DFF48029E493A3F85407240CC8C333F5
:10DE4E00C4540F4420C8834004F456800146F6DFC4
:10DE5E00E4800B010204081020408090E0AAE47ECA
:10DE6E00019360BCA3FF543F30E509541FFEE493B9
:10DE7E00A360010ECF54C025E060A840B8E493A380
:10DE8E00FAE493A3F8E493A3C8C582C8CAC583CAAB
:10DE9E00F0A3C8C582C8CAC583CADFE9DEE780BE63
:01E0DF000040
:10C95D0075F008758200EF2FFFEE33FECD33CDCC91
:10C96D0033CCC58233C5829BED9AEC99E582984014
:10C97D000CF582EE9BFEED9AFDEC99FC0FD5F0D6F1
:10C98D00E4CEFBE4CDFAE4CCF9A88222B800C1B91B
:10C99D000059BA002DEC8BF084CFCECDFCE5F0CB59
:10C9AD00F97818EF2FFFEE33FEED33FDEC33FCEB92
:10C9BD0033FB10D703994004EB99FB0FD8E5E4F94D
:10C9CD00FA227818EF2FFFEE33FEED33FDEC33FC3A
:10C9DD00C933C910D7059BE99A4007EC9BFCE99A2E
:10C9ED00F90FD8E0E4C9FAE4CCFB2275F010EF2F73
:10C9FD00FFEE33FEED33FDCC33CCC833C810D70773
:10CA0D009BEC9AE899400AED9BFDEC9AFCE899F8AD
:0ECA1D000FD5F0DAE4CDFBE4CCFAE4C8F92240
:00000001FF
